:100000000C94B7010C9414320C9441320C94DF011F
:100010000C94DF010C94DF010C94DF010C94DF01E0
:100020000C94DF010C94DF010C94DF010C94CA06E0
:100030000C94DF010C94DF010C94DF010C94DF01C0
:100040000C9420310C94DF010C9440060C947C0637
:100050000C94DF010C94DF010C94DF010C94DF01A0
:100060000C94DF010C94DF01084AD73B3BCE016EB4
:1000700084BCBFFDC12F3D6C74319ABD56833DDAFF
:100080003D00C77F11BED9E4BB4C3E916BAAAABE0E
:10009000000000803F05A84CCDB2D44EB93836A937
:1000A000020C50B9918688083CA6AAAA2ABE000074
:1000B00000803F0664EC1B3C04BC163E3BE5B93CAB
:1000C000C93C37C29E5A3D660498083EEA69AAAA0E
:1000D0003E000000803F2020BF0020BF00BF007C0A
:1000E0002020202020202020202020202020202010
:1000F00020202000C8202020202020202020202078
:1001000020C900C8202020202020202020202020BE
:10011000C97C00D820202020202020202020202042
:10012000D97C00C820202020202020202020202032
:10013000C97C00C820202020202020202020202032
:10014000C97C00207265766F006D696E6F706F7389
:1001500064206C6962726570696C6F740020202085
:100160002020BABBBCBDBE7C2020202020CACBCC26
:10017000CDCE7C00626F6F74696E672075703AED4A
:10018000F2F2F2F2F2F2F2F30062617474657279E3
:10019000207761726E696E672000747870696420E0
:1001A00076616C756573006261726F2074656D7045
:1001B0000074656D706469737020006163746976A2
:1001C000652000706173736976650075617674618E
:1001D0006C6B200073657475702073637265656E57
:1001E0007C7C7C004368617220446F6E650A00521B
:1001F0006561647920666F7220466F6E740A0055DF
:1002000070646174652043686172536574000040D6
:100210007A10F35A00A0724E18090010A5D4E80015
:1002200000E87648170000E40B54020000CA9A3B2D
:10023000000000E1F50500008096980000004042B3
:100240000F000000A0860100000010270000000041
:10025000E803000000006400000000000A00000045
:1002600000000100000000002C76D888DC674F08F1
:1002700023DFC1DFAE59E1B1B796E5E3E453C63AF7
:10028000E651997696E8E6C28426EB898C9B62ED6E
:10029000407C6FFCEFBC9C9F40F2BAA56FA5F49028
:1002A000055A2AF75C936B6CF9676DC11BFCE0E49F
:1002B0000D47FEF520E6B500D0ED902E03009435F5
:1002C00077050080841E080000204E0A000000C848
:1002D0000C333333330F986E12831141EF8D211499
:1002E000893BE65516CFFEE6DB18D1844B381BF769
:1002F0007C1D901DA4BBE424203284725E22810008
:10030000C9F124ECA1E53D276E616E00696E6600BF
:1003100000000000240027002A0000000000250043
:1003200028002B0000000000230026002900040400
:10033000040404040404020202020202030303038D
:100340000303010204081020408001020408102069
:100350000102040810200000000700020100000351
:10036000040600000000000000004B0411081124E6
:100370001FBECFEFD8E0DEBFCDBF13E0A0E0B1E0FD
:10038000E0EDFEE602C005900D92AE3FB107D9F751
:1003900016E0AEEFB3E001C01D92A43BB107E1F758
:1003A00013E0CEE6D3E004C02297FE010E9462373C
:1003B000CA36D107C9F70E942B330C9466370C94C8
:1003C0000000FA01AA27283051F1203181F1E89488
:1003D0006F936E7F6E5F7F4F8F4F9F4FAF4FB1E038
:1003E0003ED0B4E03CD0670F781F891F9A1FA11D33
:1003F000680F791F8A1F911DA11D6A0F711D811D34
:10040000911DA11D20D009F468943F912AE0269FF8
:1004100011243019305D3193DEF6CF010895462F57
:100420004770405D4193B3E00FD0C9F7F6CF462F38
:100430004F70405D4A3318F0495D31FD40524193A1
:1004400002D0A9F7EACFB4E0A6959795879577955E
:100450006795BA95C9F700976105710508959B01E5
:10046000AC010A2E06945795479537952795BA956E
:10047000C9F7620F731F841F951FA01D08952830B0
:1004800008F027E03327DA01990F311D87FD9160CD
:1004900000966105710539F432602E5F3D9330E3BB
:1004A0002A95E1F708959F3F30F080387105610586
:1004B00009F03C5F3C5F3D93913008F08068911DEE
:1004C000DF93CF931F930F93FF92EF92192F987F93
:1004D0009695E92F96959695E90FFF27E859FD4FD8
:1004E00099273327EE24FF24A701E70105900894FC
:1004F000079428F4360FE71EF81E491F511D660F9A
:10050000771F881F991F0694A1F70590079428F478
:10051000E70EF81E491F561FC11D770F881F991F30
:10052000661F0694A1F70590079428F4F80E491F5A
:10053000561FC71FD11D880F991F661F771F06946E
:10054000A1F70590079420F4490F561FC71FD81F25
:10055000990F661F771F881F0694A9F7849110953D
:10056000177041F0D695C79557954795F794E7943E
:100570001A95C1F7EEE0F2E0689415901591359167
:100580006591959105907FE27395E118F10A430B0F
:10059000560BC90BD009C0F7E10CF11E431F561FC3
:1005A000C91FD01D7EF4703311F48A95E6CFE8940C
:1005B000015030F0080F0AF40027021708F4202F2A
:1005C0002395022F7A3328F079E37D932A95E9F772
:1005D00010C07D932A9589F606949795679537956F
:1005E00017951794E118F10A430B560BC90BD00964
:1005F00098F023957E9173957A3308F070E37C939D
:100600002013B8F77E9170617D9330F0839571E38C
:100610007D9370E32A95E1F71124EF90FF900F91FD
:100620001F91CF91DF91992787FD90950895CF93E2
:10063000DF93BC018230910510F462E070E0A0917C
:10064000B206B091B306ED0140E050E0E0E0F0E02A
:1006500021C0888199818617970769F48A819B81D7
:10066000309719F09383828304C09093B3068093EC
:10067000B206FE0134C06817790738F441155105F8
:1006800019F08417950708F4AC01FE018A819B815B
:100690009C01E9012097E9F641155105A9F1CA012C
:1006A000861B970B049708F4BA01E0E0F0E02AC03B
:1006B0008D919C91119784179507F9F4641775072C
:1006C00081F412968D919C911397309719F0938332
:1006D000828304C09093B3068093B206FD013296E4
:1006E0004CC0CA01861B970BFD01E80FF91F6193EF
:1006F000719302978D939C9340C0FD0182819381F9
:100700009C01D9011097A1F68091B0069091B10695
:10071000892B41F480919F029091A0029093B106A1
:100720008093B0064091A1025091A202411551055B
:1007300041F44DB75EB780919D0290919E02481B97
:10074000590B2091B0063091B106CA01821B930B60
:100750008617970780F0AB014E5F5F4F84179507B0
:1007600050F0420F531F5093B1064093B006F90169
:100770006193719302C0E0E0F0E0CF01DF91CF918F
:100780000895CF93DF93009709F450C0EC012297AE
:100790001B821A82A091B206B091B306109709F19C
:1007A00040E050E0AC17BD0708F1BB83AA83FE010F
:1007B00021913191E20FF31FAE17BF0779F48D91AC
:1007C0009C911197280F391F2E5F3F4F3983288343
:1007D00012968D919C9113979B838A8341155105A5
:1007E00071F4D093B306C093B20620C012968D91D7
:1007F0009C911397AD01009711F0DC01D3CFFA0162
:10080000D383C28321913191E20FF31FCE17DF070B
:1008100069F488819981280F391F2E5F3F4FFA01B3
:10082000318320838A819B8193838283DF91CF915F
:100830000895FC010590615070400110D8F7809533
:1008400090958E0F9F1F0895FC016150704001909C
:100850000110D8F7809590958E0F9F1F08956EBD5B
:100860000DB407FEFDCF8EB508958DE061E00E94C6
:100870006E328BE061E00E946E328CE060E00E949C
:100880006E328AE061E00E946E321CBC80E58CBD55
:100890008DB58EB508958EEF93E00E9435040895CE
:1008A000FC011382128288EE93E0A0E0B0E0848322
:1008B0009583A683B78383EB92E091838083089529
:1008C000FC018089803419F421E030E002C020E08E
:1008D00030E0C9010895FC01818990E00895FC0190
:1008E0006487458766874787089580E090E008958C
:1008F00080E090E0089580E090E008950895EF9200
:10090000FF921F93CF93DF93162F7A0186E060E06A
:100910000E94AD328EEF93E060E00E942F048EEFD4
:1009200093E060E00E942F048EEF93E069E00E9464
:100930002F048EEF93E0612F0E942F04C0E0D0E0DF
:10094000F701EC0FFD1F10818EEF93E06AE00E942B
:100950002F048EEF93E06C2F0E942F048EEF93E014
:100960006BE00E942F048EEF93E0612F0E942F0412
:100970002196C633D10521F78EEF93E068E00E94FF
:100980002F048EEF93E060EA0E942F048EEF93E035
:1009900060EA0E942F0485FDF9CF8EEF93E060E0BE
:1009A0000E942F048EEF93E06CE00E942F0486E0FB
:1009B00061E00E94AD32DF91CF911F91FF90EF90E7
:1009C00008951F93CF93DF93EC01162F86E060E02C
:1009D0000E94AD328EEF93E060E00E942F0411235D
:1009E00019F0113059F404C08EEF93E0688904C007
:1009F00068896C618EEF93E00E942F0486E061E0CD
:100A00000E94AD32DF91CF911F910895EF92FF9236
:100A10000F931F938EE1489F70011124E60EF11C85
:100A200086E060E00E94AD320EEF13E0C80165E0A1
:100A30000E942F04C8016F2D0E942F04C80166E098
:100A40000E942F04C8016E2D0E942F041F910F9148
:100A5000FF90EF900895EF92FF920F931F937C0108
:100A60000EEF13E0C80167E00E942F04C8016FEF8A
:100A70000E942F0486E061E00E94AD32F701878575
:100A80008F5F87871F910F91FF90EF900895EF92EE
:100A9000FF920F931F93FC01E7848EE1E89E7001A3
:100AA00011248685E80EF11C86E060E00E94AD32DC
:100AB0000EEF13E0C80164E00E942F04C80163E058
:100AC0000E942F04C80165E00E942F04C8016F2D09
:100AD0000E942F04C80166E00E942F04C8016E2DF9
:100AE0000E942F041F910F91FF90EF9008951F9384
:100AF000CF93DF93EC01162F6C3731F40E942B0556
:100B0000CE010E9447050AC08EEF93E067E00E9485
:100B10002F048EEF93E0612F0E942F0481E090E07C
:100B2000DF91CF911F9108950F931F9386E060E0AE
:100B30000E94AD320EEF13E0C80164E00E942F0462
:100B4000C80164E00E942F0486E061E00E94AD329B
:100B50001F910F9108951F93CF93DF93EC01188A93
:100B600016E0198B80EA96E060E973E00E9480301D
:100B7000813049F480E4888B88E0898B86E060E0EE
:100B80000E94AD3202C0188A198B86E060E00E9494
:100B9000AD32DF91CF911F9108950F931F93CF93A3
:100BA000DF93EC0186E061E00E946E3282E060E05B
:100BB0000E946E3282E061E00E94AD32CE010E945E
:100BC000AB0586E060E00E94AD328EEF93E06CEE04
:100BD0000E942F048EEF93E06FEF0E942F04182FD6
:100BE0008EEF93E060E00E942F04688962608EEFD0
:100BF00093E00E942F0462E370E080E090E00E94A6
:100C000076318EEF93E06CE60E942F041F7E8EEF0C
:100C100093E0612F0E942F048889803419F00DE041
:100C200010E002C000E110E0109200041092FF03F7
:100C300017C06091FF0370910004605F8EEF93E036
:100C40000E942F048EEF93E069E00E942F048091B0
:100C5000FF03909100040196909300048093FF039A
:100C60008091FF03909100048017910714F3CE0147
:100C700061E00E94E104DF91CF911F910F910895EF
:100C80001F920F920FB60F9211242F933F934F9301
:100C90008F939F93EF93FF934091C60020918F060F
:100CA000309190062F5F3F4F80919306909194066C
:100CB00028233923809191069091920628173907AD
:100CC00079F080918F0690919006E0919506F091D1
:100CD0009606E80FF91F40833093900620938F0605
:100CE000FF91EF919F918F914F913F912F910F9095
:100CF0000FBE0F901F9018951F920F920FB60F9274
:100D000011242F933F938F939F93EF93FF93209101
:100D1000990630919A068091970690919806281727
:100D20003907E9F08091990690919A06E0919D0625
:100D3000F0919E06E80FF91F80818093C600809194
:100D4000990690919A06019620919B0630919C06F7
:100D50008223932390939A068093990610C0209142
:100D60009706309198068091990690919A062817D7
:100D7000390729F48091C1008F7D8093C100FF91D4
:100D8000EF919F918F913F912F910F900FBE0F90F8
:100D90001F9018951F920F920FB60F9211248F93E8
:100DA0009F938091C1049091C204892B51F080914E
:100DB000C3049091C40401969093C4048093C30427
:100DC00009C08091C5049091C60401969093C60411
:100DD0008093C5049F918F910F900FBE0F901F902D
:100DE0001895CF93DF93482FEB018091260683302F
:100DF00009F45DC0843028F48130C1F0823058F5A8
:100E00000AC0853009F4D2C0853008F4A8C0863005
:100E100009F0F2C0E9C04C3309F0EEC081E08093E4
:100E20002606488384EB80932506E6C0842F90E055
:100E3000E0912506F0E0E827F927EF53FD4F2081E8
:100E400020932506887F9070809741F582E08093FB
:100E50002606498329C0242F30E0E0912506F0E0E2
:100E6000E227F327EF53FD4F808180932506809181
:100E700024068F5F80932406823018F43B832A83F4
:100E8000BBC0922F88272A813B81820F931F9B83AF
:100E90008A830A978F3F910521F018F01092260659
:100EA000ABC083E08093260610922406A5C0E42FF1
:100EB000F0E08091250690E0E827F927EF53FD4FF9
:100EC000808180932506609124066F5F60932406DD
:100ED000623089F0633020F4613009F08DC006C0C3
:100EE000633091F0643009F087C022C0842F90E015
:100EF000A0E0B0E018C0242F30E040E050E0542FD4
:100F0000432F322F222707C0242F30E040E050E04B
:100F1000A901332722278C819D81AE81BF81820F59
:100F2000931FA41FB51F8C839D83AE83BF8364C0B2
:100F3000242F30E040E050E0522F4427332722276F
:100F40008C819D81AE81BF81820F931FA41FB51F2D
:100F50008C839D83AE83BF8360932606A5CF242F09
:100F600030E0E0912506F0E0E227F327EF53FD4F54
:100F7000808180932506809124068F5F80932406CC
:100F8000813019F08230C1F503C03987288734C019
:100F9000922F882728853985280F391F3987288778
:100FA0008A819B810A97F1F085E07CCFE42FF0E005
:100FB0008091250690E0E827F927EF53FD4F8081C7
:100FC00080932506209124062F5F2093240630E08D
:100FD000FB01E20FF31F41878A819B810A97281743
:100FE000390750F086E05ECFC75FDE4F4883C950B7
:100FF000D14087E08093260680912606873069F4E9
:1010000010922606C75FDE4F909125068881C95051
:10101000D140981711F48A8101C080E0DF91CF910F
:1010200008958F92AF92CF92EF92FF920F931F93FA
:1010300087E894E060E045EC50E024EC30E000EC20
:1010400010E0B1ECEB2EF12CCC24C394A8E9AA2E2D
:10105000F0E28F2E0E94F02984EA94E00E9450046E
:101060001092B7041092B8041092B9041092BA0406
:101070001092BB041092BC041092BD041092BE04E6
:101080001092C0041092BF041092B6041F910F91E9
:10109000FF90EF90CF90AF908F900895AF92BF9256
:1010A000CF92DF92EF92FF920F931F93E0908B0607
:1010B000F0908C0600918D0610918E068FE590E0E1
:1010C000A0E0B0E0E80EF91E0A1F1B1F0E94683165
:1010D0006E157F058007910708F44EC0A090EC04C0
:1010E000B090ED04C090EE04D090EF04C601B501BD
:1010F00020E030E040E85FE30E94CB35181694F51D
:10110000E0904306F0904406009145061091460693
:101110000E94683120918B0630918C0640918D069B
:1011200050918E06621B730B840B950B0E94A134A9
:101130009B01AC01C601B5010E94D63520E030E02C
:101140004AE754E40E9408349B01AC01C801B7018E
:101150000E943B3360934306709344068093450698
:10116000909346060E94683160938B0670938C06BC
:1011700080938D0690938E061F910F91FF90EF90B4
:10118000DF90CF90BF90AF900895DF93CF9300D0C2
:1011900000D0CDB7DEB7FB01E80FF91F628583856C
:1011A0009485258569838A839B832C83492F5C8161
:1011B000782FCA010F900F900F900F90CF91DF9171
:1011C0000895AF92BF92DF92EF92FF920F931F9319
:1011D000CF93DF938C018091270680FDE4C0F80156
:1011E000F08087E894E06F2D0E94D12AE801C75F64
:1011F000DE4FEF2DF0E0EF53FD4F80818883F80143
:10120000F18087E894E06F2D0E94D12AEF2DF0E065
:10121000888190E0E827F927EF53FD4F808188838C
:10122000F801F28087E894E06F2D0E94D12AEF2D1B
:10123000F0E0888190E0E827F927EF53FD4F8081A7
:101240008883F801F38087E894E06F2D0E94D12A0B
:10125000EF2DF0E0888190E0E827F927EF53FD4F6C
:1012600080818883F801F48087E894E06F2D0E94E4
:10127000D12AEF2DF0E0888190E0E827F927EF539D
:10128000FD4F80818883F801248135814681578113
:10129000232F342F452F5527F22E87E894E0622F15
:1012A0000E94D12AEF2DF0E0888190E0E827F9270D
:1012B000EF53FD4F80818883F80124813581468179
:1012C00057819A0144275527F22E87E894E0622F30
:1012D0000E94D12AEF2DF0E0888190E0E827F927DD
:1012E000EF53FD4F80818883F80124813581468149
:1012F0005781252F332744275527F22E87E894E07E
:10130000622F0E94D12AEF2DF0E0888190E0E8273B
:10131000F927EF53FD4F8081888387E894E060E0F0
:101320000E94D12AE881F0E0EF53FD4F808188834D
:1013300087E894E060E00E94D12AE881F0E0EF5372
:10134000FD4F80818883F801828193810B9718F18A
:101350008AE0A82EB12CA00EB11E750112C0F701B3
:10136000D1907F0187E894E06D2D0E94D12AED2D68
:10137000F0E0888190E0E827F927EF53FD4F808166
:1013800088832E2D2A1930E0F801828193810A97F3
:101390002817390720F3075F1E4F87E894E0F8010C
:1013A00060810E94D12ADF91CF911F910F91FF9010
:1013B000EF90DF90BF90AF900895DF93CF93CDB7BC
:1013C000DEB7CA50D1400FB6F894DEBF0FBECDBF16
:1013D0002CE329836A832AE030E03C832B83FC01E1
:1013E00084819581A681B7818D839E83AF83B887E1
:1013F000CE0101960E94E108C65FDE4F0FB6F89459
:10140000DEBF0FBECDBFCF91DF91089580EA96E099
:101410006AE773E00E948030882331F586E696E61D
:10142000A6E6B0E48093280690932906A0932A06A6
:10143000B0932B0680E090E0A0E8BFE380932C06F9
:1014400090932D06A0932E06B0932F0688EE93E07E
:10145000909331068093300681E8809332068DE8C0
:10146000809333068DEF25C082E598EBAEE0B0E4C3
:101470008093280690932906A0932A06B0932B0602
:1014800085E89BEEA1E5B0E480932C0690932D06B1
:10149000A0932E06B0932F0680EA94E19093310634
:1014A000809330068BEF8093320686E68093330676
:1014B0008AEF809334060895FF920F931F9300EAFA
:1014C00016E0C8016CE773E00E94803080936F06DD
:1014D000C8016EE773E00E94803080937006C801F7
:1014E00060E873E00E94803080934F06C8016EE888
:1014F00073E00E94803080936706C8016AE873E059
:101500000E94803080936506C80164E873E00E9401
:10151000803080937106C80166E873E00E948030D5
:1015200080937206C8016CE873E00E94803080935B
:101530005706C80162E973E00E9480308093730609
:10154000C80164E973E00E94803080935606C801A8
:1015500064EF73E00E948030F82EC80165EF73E0FD
:101560000E948030382F20E02F0D311D30937506FA
:1015700020937406C80166EF73E00E948030F82E55
:10158000C80167EF73E00E948030382F20E02F0DF4
:10159000311D3093770620937606C80168EF73E01B
:1015A0000E948030F82EC80169EF73E00E948030FD
:1015B000382F20E02F0D311D3093790620937806C7
:1015C000C8016BEF73E00E94803080934E061F913C
:1015D0000F91FF900895BC0180EA96E00E94803050
:1015E00008956091D6047091D7048091D8049091A9
:1015F000D90420E030E040E152E40E94D63520E0FA
:1016000030E044EB53E40E9408340E9439360E94D3
:1016100070349B012550304037FF03C09B01215E91
:101620003F4FA7E3B6E0F901EF53FC4F80818C9365
:101630002F5F3F4F2432310514F020E030E0119647
:1016400086E0A234B80779F71C9208952F923F9252
:101650004F925F926F927F928F929F92AF92BF92C2
:10166000CF92DF92EF92FF920F931F93DF93CF936E
:1016700000D000D000D0CDB7DEB7182F662E209155
:10168000CC043091CD042A35310530F0C9018D5498
:101690009F4F89359105E8F437FF02C02D543F4F25
:1016A000C90137FF03C0909581959F4F8A319105FD
:1016B0003CF0F4E48F2E912CE9ED2E2E312C1DC040
:1016C0000A975CF17BE3872E912C62ED262E312C5C
:1016D00020C02B35310514F0235B3040C90137FFA2
:1016E00003C0909581959F4F8A31910554F056E53E
:1016F000852E912C4CED242E312C37E0A32EB12CCD
:1017000015C00A9754F02DE4822E912C94ED292EC9
:10171000312C88E0A82EB12C09C005E0802E912C38
:10172000B8E32B2E312CA9E0AA2EB12C6091CE0467
:101730007091CF04882777FD8095982F0E94A3345D
:1017400027EA32E94BE25CEB0E94D6350E94AA36CA
:1017500020E030E040EA50E40E94D63520E030E05E
:1017600040E951E40E94D6350E94393620E030E04D
:1017700044E352E40E943B330E947034712EFEEB2E
:10178000CF2EFFEFDF2E9B01442737FD4095542FCE
:1017900029833A834B835C83E4EA4E2EE4E05E2E99
:1017A0004AEF5FEF240E351E6091CC047091CD049A
:1017B000882777FD8095982F0E94A33425E33AEF80
:1017C0004EE85CE30E94D6350E94AA367B018C016C
:1017D000B601882777FD8095982F0E94A3349B013E
:1017E000AC01C801B7010E94D6357B018C0169812B
:1017F0007A818B819C810E94A3349B01AC01C8013A
:10180000B7010E943B330E9470349B01CB010197CA
:101810008A35910508F071C062E170E00E941037CE
:101820008B012F5F3F4FAEEEBFEF6A9FC0016B9FF2
:10183000900D7A9F900D1124820F931F62E070E04B
:101840000E9410376D837E83E62CE01A4E2D4C5F8C
:1018500084EA94E0672D0E94060500D000D000D0F5
:10186000EDB7FEB73196ADB7BEB712965C924E9209
:10187000119720E031E0338322838D819E81880D92
:10188000991D958384830E94CF294DB75EB74A5F27
:101890005F4F0FB6F8945EBF0FBE4DBF8D819E8126
:1018A0008A159B0554F1043011053CF593E0E90ECF
:1018B000C201672D4E2D0E94060500D000D000D039
:1018C000EDB7FEB73196ADB7BEB712965C924E92A9
:1018D000119720E031E0338322834D815E81420DF8
:1018E000531D558344830E94CF298DB79EB706961A
:1018F0000FB6F8949EBF0FBE8DBFACE0B0E0CA0E2D
:10190000DB1E7394BEE4CB16D10409F04DCF2696AE
:101910000FB6F894DEBF0FBECDBFCF91DF911F9100
:101920000F91FF90EF90DF90CF90BF90AF909F907E
:101930008F907F906F905F904F903F902F90089581
:10194000823010F422E002C0282F220F30E08DB741
:101950009EB708970FB6F8949EBF0FBE8DBFEDB728
:10196000FEB7319684EA94E0ADB7BEB712969C9369
:101970008E93119783E091E09383828322573F4FA8
:10198000358324832F5F3F4F378326830E94CF29DF
:101990008DB79EB708960FB6F8949EBF0FBE8DBF49
:1019A0000895CF93DF93AC01E091DE04F091DF0462
:1019B0002091350630913606C9018C599F4F8E17FC
:1019C0009F071CF4EA01219709C024563040E21712
:1019D000F30714F0EA0102C0EA012196842F90E097
:1019E000C817D90729F080EA96E04C2F0E9487306B
:1019F000CE01DF91CF9108950F931F9300EA16E077
:101A0000C80163EF73E041E00E948730C80164EFD2
:101A100073E043E10E948730C80165EF73E046E060
:101A20000E948730C80166EF73E040E10E94873072
:101A3000C80167EF73E047E20E948730C80168EF92
:101A400073E048E80E948730C80169EF73E043E122
:101A50000E9487301F910F910895CF92DF92EF92ED
:101A6000FF920F931F937C01D62EC72E04EA14E039
:101A7000C8016E2D4D2D0E946F04C8010E944705BC
:101A800000D000D0EDB7FEB71283018383E391E06D
:101A9000948383830E94BE29EDB7FEB7128301832E
:101AA00083E291E0948383830E94BE29EDB7FEB761
:101AB0001283018383E191E0948383830E94BE2992
:101AC000EDB7FEB71283018383E091E094838383B3
:101AD0000E94BE29EDB7FEB71283018384EF90E028
:101AE000948383830E94BE290F900F900F900F90D4
:101AF000C8010E942B05C70101966D2D7C2D0E9407
:101B0000260B1F910F91FF90EF90DF90CF900895DB
:101B1000CF92DF92EF92FF920F931F93CF93DF93B9
:101B2000182F062F0E94683128EE33E040E050E085
:101B30000E94233769017A01C4EAD4E0CE01612F03
:101B4000402F0E946F04CE010E9447058091FE0441
:101B50009091FF04892B09F453C000910005109166
:101B600001058DB79EB744970FB6F8949EBF0FBE80
:101B70008DBFEDB7FEB73196ADB7BEB71296DC9309
:101B8000CE93119788E091E09383828383EB90E07A
:101B900095838483C6016CE370E00E941037CB010B
:101BA0006CE370E00E941037978386832AE330E06D
:101BB00031872087C6016CE370E00E94103793875D
:101BC000828785E690E095878487C8016CE370E0A2
:101BD0000E94FC36CB016CE370E00E9410379787BF
:101BE0008687318B208BC8016CE370E00E94FC3645
:101BF000938B828B0E94CF298DB79EB7449633C0BA
:101C0000ADB7BEB71C970FB6F894BEBF0FBEADBF41
:101C1000EDB7FEB731961296DC93CE93119780E222
:101C200091E09383828383EB90E095838483C60164
:101C30006CE370E00E941037CB016CE370E00E940F
:101C40001037978386838AE390E091878087C60167
:101C50006CE370E00E941037938782870E94CF293F
:101C60008DB79EB70C960FB6F8949EBF0FBE8DBF72
:101C700084EA94E00E942B05DF91CF911F910F9190
:101C8000FF90EF90DF90CF900895EF92FF920F9327
:101C90001F93282F462FA4EAEA2EA4E0FA2EC701AC
:101CA000622F0E946F04C7010E9447058DB79EB73F
:101CB0000A970FB6F8949EBF0FBE8DBF0DB71EB723
:101CC0000F5F1F4FEDB7FEB7F282E1828CE291E029
:101CD000F8019383828360910205709103058091DE
:101CE00004059091050520912C0630912D06409118
:101CF0002E0650912F060E94D635F8016483758315
:101D00008683978380EB90E0918780870E94CF291C
:101D10008DB79EB70A960FB6F8949EBF0FBE8DBFC3
:101D2000C7010E942B051F910F91FF90EF9008951E
:101D30008F929F92AF92BF92CF92DF92EF92FF92DB
:101D40000F931F93E82EF62E04EA14E0C8016E2DBF
:101D50004F2D0E946F04C8010E9447058DB79EB7A2
:101D60000C970FB6F8949EBF0FBE8DBFEDB7FEB7B0
:101D70003196ADB7BEB712961C930E93119794E3AC
:101D8000892E91E0992E938282828DEEA82EB12C1D
:101D9000B582A48280910B0590910C05A0910D0550
:101DA000B0910E0586839783A087B187B3EFCB2EC2
:101DB000D12CD386C2860E94CF298DB79EB70C96B0
:101DC0000FB6F8949EBF0FBE8DBFC8010E942B05B1
:101DD000F394C8016E2D4F2D0E946F04C8010E941C
:101DE0004705ADB7BEB71C970FB6F894BEBF0FBE80
:101DF000ADBFEDB7FEB7319612961C930E931197B7
:101E000093828282B582A48280910F059091100501
:101E1000A0911105B091120586839783A087B187A1
:101E2000D386C2860E94CF298DB79EB70C960FB677
:101E3000F8949EBF0FBE8DBFC8010E942B05F3947E
:101E4000C8016E2D4F2D0E946F04C8010E944705E6
:101E5000ADB7BEB71C970FB6F894BEBF0FBEADBFEF
:101E6000EDB7FEB7319612961C930E93119793829D
:101E70008282B582A4828091130590911405A0916D
:101E80001505B091160586839783A087B187D38601
:101E9000C2860E94CF298DB79EB70C960FB6F894D4
:101EA0009EBF0FBE8DBFC8010E942B051F910F91D1
:101EB000FF90EF90DF90CF90BF90AF909F908F906A
:101EC00008950F931F93282F462F04EA14E0C801AA
:101ED000622F0E946F04C8010E9447058DB79EB70C
:101EE0000A970FB6F8949EBF0FBE8DBFEDB7FEB731
:101EF0003196ADB7BEB712961C930E9311978EE331
:101F000091E09383828389EB90E095838483809131
:101F1000FE049091FF049783868382E890E0918786
:101F200080870E94CF298DB79EB70A960FB6F89486
:101F30009EBF0FBE8DBFC8010E942B051F910F9140
:101F40000895EF92FF920F931F93282F462F34EAA4
:101F5000E32E34E0F32EC701622F0E946F04C70105
:101F60000E9447058DB79EB70C970FB6F8949EBF99
:101F70000FBE8DBF0DB71EB70F5F1F4FEDB7FEB77A
:101F8000F282E18286E491E0F8019383828384EE19
:101F900090E0958384836091FC047091FD04882710
:101FA00077FD8095982F0E94A3342AE037ED43E215
:101FB0005CE30E94D635F80166837783808791873A
:101FC0008FE890E0938782870E94CF298DB79EB7D4
:101FD0000C960FB6F8949EBF0FBE8DBFC7010E942E
:101FE0002B051F910F91FF90EF9008950F931F9372
:101FF000282F462F04EA14E0C801622F0E946F04C4
:10200000C8010E9447058DB79EB70C970FB6F8948C
:102010009EBF0FBE8DBFEDB7FEB73196ADB7BEB751
:1020200012961C930E93119786E491E0938382831A
:1020300082EE90E0958384838091F8049091F90476
:10204000A091FA04B091FB0486839783A087B1879F
:102050008EE890E0938782870E94CF298DB79EB744
:102060000C960FB6F8949EBF0FBE8DBFC8010E949C
:102070002B051F910F9108950F931F93282F462F23
:1020800084EA94E0622F0E946F0484EA94E00E9444
:1020900047058091DB04882319F420E531E057C01F
:1020A000813019F424E531E052C0823019F428E57A
:1020B00031E04DC0833019F42CE531E048C0843064
:1020C00019F420E631E043C0853019F424E631E00C
:1020D0003EC0863019F428E631E039C0873019F463
:1020E0002CE631E034C0883019F420E731E02FC00D
:1020F000893019F424E731E02AC08A3019F428E73E
:1021000031E025C08B3019F42CE731E020C08C3051
:1021100019F420E831E01BC08D3019F424E831E0D7
:1021200016C08E3019F428E831E011C08F3019F450
:102130002CE831E00CC0803119F420E931E007C00F
:10214000813119F024E931E002C025E931E08DB791
:102150009EB708970FB6F8949EBF0FBE8DBFEDB720
:10216000FEB7319604EA14E0ADB7BEB712961C93E1
:102170000E93119789E991E09383828380EE90E03A
:1021800095838483378326830E94CF298DB79EB79A
:1021900008960FB6F8949EBF0FBE8DBFC8010E946F
:1021A0002B051F910F9108950F931F93282F462FF2
:1021B00004EA14E0C801622F0E946F04C8010E9463
:1021C00047058DB79EB70A970FB6F8949EBF0FBE0E
:1021D0008DBFEDB7FEB73196ADB7BEB712961C9363
:1021E0000E9311978EE991E09383828387E890E0C4
:1021F000958384838091DC049091DD0497838683AA
:1022000085E290E0918780870E94CF298DB79EB7A5
:102210000A960FB6F8949EBF0FBE8DBFC8010E94EC
:102220002B051F910F9108950F931F93282F462F71
:1022300004EA14E0C801622F0E946F04C8010E94E2
:1022400047058DB79EB70A970FB6F8949EBF0FBE8D
:102250008DBFEDB7FEB73196ADB7BEB712961C93E2
:102260000E93119788EA91E0938382838091CE0444
:102270009091CF049583848380EB90E0978386834D
:1022800081EB90E0918780870E94CF298DB79EB720
:102290000A960FB6F8949EBF0FBE8DBFC8010E946C
:1022A0002B051F910F9108950F931F93282F462FF1
:1022B00004EA14E0C801622F0E946F04C8010E9462
:1022C00047058DB79EB70A970FB6F8949EBF0FBE0D
:1022D0008DBFEDB7FEB73196ADB7BEB712961C9362
:1022E0000E93119788EA91E0938382838091CC04C6
:1022F0009091CD049583848380EB90E097838683CF
:1023000082EB90E0918780870E94CF298DB79EB79E
:102310000A960FB6F8949EBF0FBE8DBFC8010E94EB
:102320002B051F910F9108950F931F93282F462F70
:1023300004EA14E0C801622F0E946F04C8010E94E1
:1023400047058DB79EB70A970FB6F8949EBF0FBE8C
:102350008DBFEDB7FEB73196ADB7BEB712961C93E1
:102360000E93119780EB91E09383828381EE90E04E
:10237000958384838091AB029091AC02978386838E
:1023800085E290E0918780870E94CF298DB79EB724
:102390000A960FB6F8949EBF0FBE8DBFC8010E946B
:1023A0002B051F910F9108950F931F93282F462FF0
:1023B00004EA14E0C801622F0E946F04C8010E9461
:1023C00047058DB79EB70C970FB6F8949EBF0FBE0A
:1023D0008DBFEDB7FEB73196ADB7BEB712961C9361
:1023E0000E93119788EB91E09383828382EC91E0C6
:1023F0009583848380ED90E09783868387E396E0DE
:102400009187808781ED90E0938782870E94CF2912
:102410008DB79EB70C960FB6F8949EBF0FBE8DBFBA
:10242000C8010E942B051F910F9108950F931F93D0
:10243000282F462F04EA14E0C801622F0E946F047F
:10244000C8010E9447058DB79EB70A970FB6F8944A
:102450009EBF0FBE8DBFEDB7FEB73196ADB7BEB70D
:1024600012961C930E93119780ED91E093838283D3
:102470008091D6049091D704A091D804B091D9044A
:1024800084839583A683B78380EB90E091878087D0
:102490000E94CF298DB79EB70A960FB6F8949EBFBB
:1024A0000FBE8DBFC8010E942B051F910F9108958B
:1024B0000F931F93282F462F04EA14E0C801622FC0
:1024C0000E946F04C8010E9447058DB79EB70C9704
:1024D0000FB6F8949EBF0FBE8DBFEDB7FEB7319615
:1024E000ADB7BEB712961C930E93119788ED91E08D
:1024F0009383828386E190E0958384838091F004C6
:102500009091F104A091F204B091F3048683978333
:10251000A087B18788E890E0938782870E94CF29BF
:102520008DB79EB70C960FB6F8949EBF0FBE8DBFA9
:10253000C8010E942B051F910F910895CF92DF9241
:10254000EF92FF920F931F93CF93DF93282F462F85
:10255000C4EAD4E0CE01622F0E946F04CE010E9433
:10256000470560914306709144068091450690911D
:10257000460620912C0630912D0640912E06509152
:102580002F060E94D6356B017C0120E030E04AE73F
:1025900054E40E94CB351816D4F58DB79EB70C972E
:1025A0000FB6F8949EBF0FBE8DBF0DB71EB70F5F5D
:1025B0001F4FADB7BEB71296DC93CE93119786E44A
:1025C00091E0F801938382838EEF90E0958384837A
:1025D0006091300670913106882777FD8095982F9D
:1025E0000E94A3349B01AC01C701B6010E940834CC
:1025F000D80116966D937D938D939C931997809136
:1026000034061A968C931A971B961C9221C08DB78C
:102610009EB70C970FB6F8949EBF0FBE8DBFEDB757
:10262000FEB73196ADB7BEB71296DC93CE93119735
:1026300082EE91E0938382838EEF90E09583848392
:10264000C682D782E086F186809133068287138620
:102650000E94CF29EDB7FEB73C960FB6F894FEBFA7
:102660000FBEEDBF84EA94E00E942B05DF91CF916D
:102670001F910F91FF90EF90DF90CF900895EF9210
:10268000FF920F931F93282F462F54EAE52E54E014
:10269000F52EC701622F0E946F04C7010E944705F3
:1026A0008DB79EB70C970FB6F8949EBF0FBE8DBF27
:1026B0000DB71EB70F5F1F4FEDB7FEB7F282E18275
:1026C00088ED91E0F8019383828389EE90E0958311
:1026D00084836091EC047091ED048091EE049091FC
:1026E000EF04209128063091290640912A06509146
:1026F0002B060E94D635F801668377838087918701
:1027000080913206828713860E94CF298DB79EB7AB
:102710000C960FB6F8949EBF0FBE8DBFC7010E94E6
:102720002B051F910F91FF90EF900895EF92FF926C
:102730000F931F93282F462F64EAE62E64E0F62EAF
:10274000C701622F0E946F04C7010E9447058DB721
:102750009EB70C970FB6F8949EBF0FBE8DBF0DB7F6
:102760001EB70F5F1F4FEDB7FEB7F282E18288ED13
:1027700091E0F8019383828388EE90E095838483CF
:102780006091F4047091F5048091F6049091F7043F
:10279000209128063091290640912A0650912B0657
:1027A0000E94D635F8016683778380879187809170
:1027B0003206828713860E94CF298DB79EB70C966A
:1027C0000FB6F8949EBF0FBE8DBFC7010E942B05A8
:1027D0001F910F91FF90EF900895EF92FF920F934A
:1027E0001F93282F462F74EAE72E74E0F72EC701B7
:1027F000622F0E946F04C7010E9447058DB79EB7E4
:102800000C970FB6F8949EBF0FBE8DBF0DB71EB7C5
:102810000F5F1F4FEDB7FEB7F282E18282EE91E0CB
:10282000F8019383828386EE90E0958384836091A0
:10283000E8047091E9048091EA049091EB042091FE
:102840002C0630912D0640912E0650912F060E94A5
:10285000D635F80166837783808791878091330628
:10286000828713860E94CF298DB79EB70C960FB62C
:10287000F8949EBF0FBE8DBFC7010E942B051F910C
:102880000F91FF90EF900895EF92FF920F931F9397
:10289000282F462FE4EAEE2EE4E0FE2EC701622F39
:1028A0000E946F04C7010E9447058DB79EB70C9721
:1028B0000FB6F8949EBF0FBE8DBF0DB71EB70F5F4A
:1028C0001F4FEDB7FEB7F282E18282EE91E0F80190
:1028D0009383828387EE90E09583848360910605DD
:1028E00070910705882777FD8095982F0E94A33463
:1028F00020912C0630912D0640912E0650912F06E6
:102900000E94D635F801668377838087918780910E
:102910003306828713860E94CF298DB79EB70C9607
:102920000FB6F8949EBF0FBE8DBFC7010E942B0546
:102930001F910F91FF90EF9008950F931F93282FF1
:10294000462F04EA14E0C801622F0E946F04C801F8
:102950000E944705809147060E94A00CC8010E9472
:102960002B051F910F910895EF92FF920F931F93E4
:10297000282F462FF4EAEF2EF4E0FF2EC701622F36
:102980000E946F04C7010E9447058DB79EB70C9740
:102990000FB6F8949EBF0FBE8DBF0DB71EB70F5F69
:1029A0001F4FEDB7FEB7F282E18282EE91E0F801AF
:1029B000938382838FE190E09583848360914806BE
:1029C0007091490680914A0690914B060E94A3346B
:1029D00020912C0630912D0640912E0650912F0605
:1029E0000E94D635F801668377838087918780912E
:1029F0003306828713860E94CF298DB79EB70C9627
:102A00000FB6F8949EBF0FBE8DBFC7010E942B0565
:102A10001F910F91FF90EF9008950F931F93282F10
:102A2000462F04EA14E0C801622F0E946F04C80117
:102A30000E9447058DB79EB740970FB6F8949EBF8A
:102A40000FBE8DBFEDB7FEB73196ADB7BEB71296CC
:102A50001C930E9311978CEE91E09383828383E80D
:102A600090E0958384838091D2049091D304A091C7
:102A7000D404B091D50486839783A087B18784E876
:102A800090E0938782878091E2049091E304A09183
:102A9000E404B091E50484879587A687B7870E94F0
:102AA000CF298DB79EB740960FB6F8949EBF0FBE44
:102AB0008DBFC8010E942B051F910F9108950F93A0
:102AC0001F93282F462F84EA94E0622F0E946F0400
:102AD00084EA94E00E9447058091E704282F30E0C3
:102AE000823030F4A4E0220F331FAA95E1F702C030
:102AF0002150304000D000D000D0EDB7FEB7319665
:102B000004EA14E0ADB7BEB712961C930E9311976A
:102B100080E091E093838283358324830E94CF29D0
:102B20008DB79EB706960FB6F8949EBF0FBE8DBFA9
:102B3000C8010E942B051F910F9108950F931F93B9
:102B4000282F462F04EA14E0C801622F0E946F0468
:102B5000C8010E9447058DB79EB708970FB6F89435
:102B60009EBF0FBE8DBFEDB7FEB73196ADB7BEB7F6
:102B700012961C930E9311978EEF91E093838283AC
:102B80008FE090E0958384838091E60486831782AA
:102B90000E94CF298DB79EB708960FB6F8949EBFB6
:102BA0000FBE8DBFC8010E942B051F910F91089584
:102BB0000F931F9304EA14E0C80163E045E00E940C
:102BC0006F04C8010E94470500D000D0EDB7FEB7E2
:102BD000128301838DE591E0948383830E94BE2953
:102BE000EDB7FEB71283018389E491E09483838378
:102BF0000E94BE29EDB7FEB71283018383E491E002
:102C0000948383830E94BE290F900F900F900F90A2
:102C1000C8010E942B051F910F9108950F931F93D8
:102C2000282F462F04EA14E0C801622F0E946F0487
:102C3000C8010E94470500D000D0EDB7FEB712834F
:102C4000018384E791E0948383830E94BE290F90DF
:102C50000F900F900F90C8010E942B051F910F91AC
:102C60000895EF92FF920F931F93CF93DF930E94EB
:102C7000683120915106309152064091530650918F
:102C80005406261737074807590708F08AC10E94DB
:102C900068316C507E4F8F4F9F4F609351067093F9
:102CA0005206809353069093540604EA14E0C80138
:102CB0000E949405C80165E043E00E946F04C801CA
:102CC0000E94470500D000D0EDB7FEB71283018304
:102CD00084ED91E0948383830E94BE290F900F902E
:102CE0000F900F908091350690913606892B31F028
:102CF00080914C0690914D06892B81F48091DE04E1
:102D00009091DF0490933606809335068091E0041D
:102D10009091E10490934D0680934C062091E0043D
:102D20003091E10440914C0650914D06C901845602
:102D300090404817590724F4809150068F5F08C0CF
:102D40002C593F4F241735072CF4809150068150A1
:102D50008093500680915006181614F081E003C04D
:102D600084301CF083E080935006809150068230BE
:102D700009F462C0833009F4BEC0813009F00DC18E
:102D800000D000D0C4EAD4E0EDB7FEB7D283C1834F
:102D90008BEC91E0948383830E94BE298091270667
:102DA0000F900F900F900F9080FF22C000D000D0A6
:102DB000EDB7FEB7D283C18383EC91E09483838324
:102DC0000E94BE2980913506909136068456904027
:102DD0000F900F900F900F902091DE043091DF0440
:102DE000281739070CF0D9C0809127068E7F21C0A3
:102DF00000D000D0EDB7FEB7D283C1838BEB91E05A
:102E0000948383830E94BE29809135069091360673
:102E10008C599F4F0F900F900F900F902091DE04D0
:102E20003091DF04821793070CF0B7C0809127061A
:102E3000816080932706B1C000D000D0C4EAD4E0FE
:102E4000EDB7FEB7D283C18381EB91E09483838396
:102E50000E94BE290F900F900F900F9080914E0608
:102E6000882301F100D000D0EDB7FEB7D283C18333
:102E700087EA91E0948383830E94BE29809135067E
:102E800090913606845690400F900F900F900F90BF
:102E90002091DE043091DF04281739071CF51092C9
:102EA0004E0620C000D000D0EDB7FEB7D283C1835C
:102EB0008AE991E0948383830E94BE29809135063C
:102EC000909136068C599F4F0F900F900F900F9056
:102ED0002091DE043091DF04821793071CF481E017
:102EE00080934E0680EA96E06BEF73E040914E06C9
:102EF0000E94873052C000D000D0B4EAEB2EB4E07C
:102F0000FB2EEDB7FEB7F282E18289E891E094836F
:102F100083830E94BE298DB79EB708970FB6F89499
:102F20009EBF0FBE8DBF0DB71EB70F5F1F4FEDB712
:102F3000FEB7F282E18284E092E0F801938382831B
:102F400060914F0670E080E090E00E94A13420E0A4
:102F500030E040E251E40E940834F8016483758354
:102F60008683978386E790E09187808780E290E070
:102F7000938782870E94CF298DB79EB70C960FB694
:102F8000F8949EBF0FBE8DBF80914F0690E060E821
:102F900073E00E94D10C80934F0684EA94E00E9473
:102FA0002B05DF91CF911F910F91FF90EF90089526
:102FB000BF92CF92DF92EF92FF920F931F93CF9326
:102FC000DF93E82ED62E0E94683120915E06309164
:102FD0005F06409160065091610626173707480743
:102FE000590708F024C1809162068823C9F08093B4
:102FF000AD02109262068CE092E09093640680939A
:1030000063060E9468316C507E4F8F4F9F4F6093D4
:103010005E0670935F068093600690936106C2C05F
:103020008091AD02A82FB0E07091DA044091630660
:1030300050916406F090C7041091E7040091550682
:1030400060911805E091AB02F091AC0280915606B8
:10305000C82FD0E0B0905706909117059D012F5FC3
:103060003F4F273031051CF021E030E019C02330FC
:10307000310531F12430310544F42130310581F03E
:103080002230310509F057C012C02530310591F1C9
:1030900025303105ECF02630310509F04CC037C041
:1030A000723008F048C049E152E081E049C083E055
:1030B000C82EFC1409F43FC046E252E082E040C052
:1030C0001230C8F50023B9F143E352E083E038C081
:1030D000623088F1633039F0643041F0623041F49D
:1030E00040E452E005C04DE452E002C04AE552E03F
:1030F00084E026C0EC17FD07F4F48FEFED39F807F4
:10310000D1F0BB20C1F447E652E085E019C072302F
:1031100090F4923080F0933039F0943041F0923056
:1031200051F444E752E005C040E852E002C04DE8E7
:1031300052E086E005C02A173B0709F090CF60C037
:1031400050936406409363068093620681E0809307
:1031500058060E94683168517C4F8F4F9F4F609393
:103160005E0670935F0680936006909361060E94EE
:1031700068316056704F8F4F9F4F60935A0670931F
:103180005B0680935C0690935D06809159068823C8
:1031900021F084EA94E00E9494051092590602C03E
:1031A0001092580604EA14E0C8016E2D4D2D0E94BD
:1031B0006F04C8010E94470500D000D000D0EDB7D1
:1031C000FEB73196ADB7BEB712961C930E9311970A
:1031D0008AE992E0938382838091630690916406EA
:1031E000958384830E94CF298DB79EB706960FB62C
:1031F000F8949EBF0FBE8DBFC8010E942B0517C05B
:103200005093640640936306109262060E946831F0
:1032100020915A0630915B0640915C0650915D0604
:10322000261737074807590708F4BACFBBCFDF91F5
:10323000CF911F910F91FF90EF90DF90CF90BF90B3
:103240000895EF92FF920F931F938091650684304B
:1032500009F056C09091DB04943008F027C18091AA
:103260006E068917A1F190936E060E9468316093F3
:103270006A0670936B0680936C0690936D0690912E
:103280006E068091AE02981711F580915906813033
:1032900091F0813018F08230B1F413C011E0109336
:1032A00059060E946831615375478040904030F460
:1032B0001093660608C082E0809359061092660655
:1032C00002C01092590684EA94E00E9494050E947C
:1032D000683120916A0630916B0640916C065091DE
:1032E0006D06621B730B840B950B615D774080400C
:1032F000904008F4DBC08091DB048093AE02D6C01E
:10330000853029F48091A3029091A40214C08630E4
:1033100029F48091A5029091A6020DC0873029F46E
:103320008091A7029091A80206C0883041F4809154
:10333000A9029091AA0290936906809368068091F1
:1033400067062091680630916906882309F04AC013
:10335000C901895097408F5A9440C8F40E9468313F
:10336000615375478040904020F481E08093660669
:103370000CC080916606882341F48091580688230A
:1033800021F484EA94E00E94940582E028C044E09D
:10339000203B340768F480915906882349F0109245
:1033A000660684EA94E00E949405109259067EC055
:1033B000205B34402955324008F078C0809159068E
:1033C000813009F473C080915806882309F06EC0DB
:1033D0001092660684EA94E00E94940581E080934E
:1033E000590664C0215B344008F460C00E94683113
:1033F000615375478040904008F041C08091660657
:103400008823E9F5E0906A06F0906B0600916C065F
:1034100010916D0688EE93E0A0E0B0E0E80EF91E92
:103420000A1F1B1F0E946831E616F70608071907D6
:10343000E8F581E08093660617C01092660684EA7C
:1034400094E00E94940580915906823019F41092FC
:10345000590603C08F5F80935906809159068230C8
:1034600018F082E0809359060E94683160936A06E2
:1034700070936B0680936C0690936D0617C0E09076
:103480006A06F0906B0600916C0610916D0688EE4E
:1034900093E0A0E0B0E0E80EF91E0A1F1B1F0E9497
:1034A0006831E616F7060807190738F21F910F91E1
:1034B000FF90EF90089580916506843010F00E948F
:1034C000211980916606882319F00E94311608950B
:1034D0008091070480FF08C060916D0480916B04A7
:1034E00090E070E00E94D81780915906823008F071
:1034F00012C2A82FB0E0FD01EF5FFB4F808185FF76
:103500000BC0FD01E35EFB4F6081A55EBB4F8C915C
:1035100090E070E00E949E1580915906A82FB0E0BF
:10352000FD01EF5FFB4F808186FF0BC0FD01EF5D6A
:10353000FB4F6081A15EBB4F8C9190E070E00E94D8
:103540005F1580915506882309F43FC08091590684
:10355000A82FB0E0FD01EF5FFB4F808187FF0BC01C
:10356000FD01EB5DFB4F6081AD5DBB4F8C9190E049
:1035700070E00E940D1580915906A82FB0E0FD0162
:10358000ED5FFB4F808184FF0BC0FD01E35CFB4FCF
:103590006081A55CBB4F8C9190E070E00E94B414F8
:1035A00080915906A82FB0E0FD01ED5FFB4F8081AF
:1035B00083FF0BC0FD01E75CFB4F6081A95CBB4F43
:1035C0008C9190E070E00E949D1480915906A82F84
:1035D000B0E0FD01EB5FFB4F808187FF0BC0FD0179
:1035E000EB5AFB4F6081AD5ABB4F8C9190E070E07D
:1035F0000E94441480915906A82FB0E0FD01E95FB4
:10360000FB4F808183FF0BC0FD01EB58FB4F6081B6
:10361000AD58BB4F8C9190E070E00E9458128091A1
:103620005906A82FB0E0FD01EB5FFB4F808181FFC1
:103630000BC0FD01E35AFB4F6081A55ABB4F8C9133
:1036400090E070E00E94961380915506882309F45B
:1036500044C08091E704823008F43FC0809159064D
:10366000A82FB0E0FD01E75FFB4F808182FF0BC018
:10367000FD01EF57FB4F6081A158BB4F8C9190E04B
:1036800070E00E949E1280915906A82FB0E0FD01C3
:10369000EB5FFB4F808182FF0BC0FD01EF5AFB4FB8
:1036A0006081A15BBB4F8C9190E070E00E94ED13B4
:1036B00080915906A82FB0E0FD01EB5FFB4F8081A0
:1036C00083FF0BC0FD01E75AFB4F6081A95ABB4F36
:1036D0008C9190E070E00E943F1380915906A82FD2
:1036E000B0E0FD01ED5FFB4F808181FF0BC0FD016C
:1036F000EF5CFB4F6081A15DBB4F8C9190E070E06F
:103700000E94161280915906A82FB0E0FD01ED5FCE
:10371000FB4F808180FF0BC0FD01E35DFB4F6081AB
:10372000A55DBB4F8C9190E070E00E94D411809118
:103730005906A82FB0E0FD01E95FFB4F808186FFAD
:103740000BC0FD01E358FB4F6081A558BB4F8C9126
:1037500090E070E00E94941180915906A82FB0E08B
:10376000FD01EF5FFB4F808182FF0BC0FD01EB5E2F
:10377000FB4F6081AD5EBB4F8C9190E070E00E948A
:10378000541180915906A82FB0E0FD01EF5FFB4F67
:10379000808181FF0BC0FD01EF5EFB4F6081A15F67
:1037A000BB4F8C9190E070E00E94141180915906FB
:1037B000A82FB0E0FD01EB5FFB4F808184FF0BC0C1
:1037C000FD01EF59FB4F6081A15ABB4F8C9190E0F6
:1037D00070E00E94D41080915906A82FB0E0FD013E
:1037E000EB5FFB4F808185FF0BC0FD01EB59FB4F69
:1037F0006081AD59BB4F8C9190E070E00E943C100D
:1038000080915906A82FB0E0FD01EF5FFB4F80814A
:1038100083FF0BC0FD01E75EFB4F6081A95EBB4FDC
:103820008C9190E070E00E94F60F80915906A82FCD
:10383000B0E0FD01EB5FFB4F808180FF0BC0FD011D
:10384000E35BFB4F6081A55BBB4F8C9190E070E028
:103850000E94A10F80915906A82FB0E0FD01EF5FF3
:10386000FB4F808184FF0BC0FD01E75DFB4F608152
:10387000A95DBB4F8C9190E070E00E94610F809138
:103880005906A82FB0E0FD01E75FFB4F808181FF63
:1038900018C080914E06FD01ED57FB4F813049F471
:1038A000AB57BB4F6C91808190E070E00E94450E59
:1038B00008C0AB57BB4F6C91808190E070E00E94D4
:1038C000980E80915906A82FB0E0FD01ED5FFB4FE7
:1038D000808187FF0BC0FD01E75BFB4F6081A95B27
:1038E000BB4F8C9190E070E00E94880D809159064A
:1038F000A82FB0E0FD01EB5FFB4F808186FF0BC07E
:10390000FD01E759FB4F6081A959BB4F8C9190E0B5
:1039100070E00E942D0D089584EA94E00E949405C1
:103920000E94D8150E94060A0895CF93DF93EC01F8
:1039300084EA94E00E946B04C817D9073CF084EA3B
:1039400094E00E946004892B09F42397CE01DF9153
:10395000CF910895EF92FF920F931F93CF93DF9330
:103960000091590610E08AEF90E0089F7001099FCE
:10397000F00C189FF00C1124C7010E94EB0AF8010B
:10398000EF5FFB4F882319F08081816002C0808146
:103990008E7F808380915906C82FD0E0C7010296A0
:1039A0000E94EB0AC55FDB4F888380915906C82FC0
:1039B000D0E0C70104960E94EB0A90E00E94951C9B
:1039C000C35FDB4F88830091590610E0C70188561A
:1039D0009F4F0E94EB0AF801EF5FFB4F882319F01D
:1039E0008081806102C080818F7E808380915906B2
:1039F000C82FD0E0C70186569F4F0E94EB0AC95DD1
:103A0000DB4F888380915906C82FD0E0C7018456C8
:103A10009F4F0E94EB0A90E00E94951CC75DDB4F10
:103A200088830091590610E0C70106960E94EB0AB0
:103A3000F801EF5FFB4F882319F08081826002C09C
:103A400080818D7F808380915906C82FD0E0C70187
:103A500008960E94EB0AC15FDB4F8883809159066C
:103A6000C82FD0E0C7010A960E94EB0A90E00E949E
:103A7000951CCF5EDB4F88830091590610E0C7018B
:103A80000C960E94EB0AF801EF5FFB4F882319F0B8
:103A90008081846002C080818B7F80838091590601
:103AA000C82FD0E0C7010E960E94EB0ACD5EDB4F17
:103AB000888380915906C82FD0E0C70140960E94A4
:103AC000EB0A90E00E94951CCB5EDB4F888300914F
:103AD000590610E0C70142960E94EB0AF801EF5F19
:103AE000FB4F882319F08081886002C08081877F26
:103AF000808380915906C82FD0E0C70144960E9468
:103B0000EB0AC95EDB4F888380915906C82FD0E04D
:103B1000C70146960E94EB0A90E00E94951CC75E82
:103B2000DB4F88830091590610E0C7014E960E9432
:103B3000EB0AF801EF5FFB4F882319F08081806268
:103B400002C080818F7D808380915906C82FD0E08C
:103B5000C70180960E94EB0AC55EDB4F8883809187
:103B60005906C82FD0E0C70182960E94EB0A90E068
:103B70000E94951CC35EDB4F88830091590610E0BC
:103B8000C70184960E94EB0AF801EF5FFB4F882380
:103B900019F08081806402C080818F7B8083809156
:103BA0005906C82FD0E0C70186960E94EB0AC15E75
:103BB000DB4F888380915906C82FD0E0C7018896D3
:103BC0000E94EB0A90E00E94951CCF5DDB4F88833A
:103BD0000091590610E0C7018A960E94EB0AF8018D
:103BE000EF5FFB4F882319F08081806802C08081DD
:103BF0008F77808380915906C82FD0E0C7018C96BB
:103C00000E94EB0ACD5DDB4F888380915906C82F57
:103C1000D0E0C7018E960E94EB0A90E00E94951CAE
:103C2000CB5DDB4F88830091590610E0C701C09639
:103C30000E94EB0AF801ED5FFB4F882319F08081A9
:103C4000816002C080818E7F808380915906C82F59
:103C5000D0E0C701C2960E94EB0AC55DDB4F8883A6
:103C600080915906C82FD0E0C701C4960E94EB0A84
:103C700090E00E94951CC35DDB4F8883009159063C
:103C800010E0C701C6960E94EB0AF801ED5FFB4FFA
:103C9000882319F08081826002C080818D7F8083BB
:103CA00080915906C82FD0E0C701C8960E94EB0A40
:103CB000C15DDB4F888380915906C82FD0E0C701D2
:103CC000CA960E94EB0A90E00E94951CCF5CDB4FE5
:103CD00088830091590610E0C701CC960E94EB0A38
:103CE000F801ED5FFB4F882319F08081846002C0EA
:103CF00080818B7F808380915906C82FD0E0C701D7
:103D0000CE960E94EB0ACD5CDB4F888380915906EA
:103D1000C82FD0E0C701805C9F4F0E94EB0A90E063
:103D20000E94951CCB5CDB4F88830091590610E004
:103D3000C701885B9F4F0E94EB0AF801ED5FFB4FC4
:103D4000882319F08081806102C080818F7E80830A
:103D500080915906C82FD0E0C701865B9F4F0E9413
:103D6000EB0AC55CDB4F888380915906C82FD0E0F1
:103D7000C701845B9F4F0E94EB0A90E00E94951C54
:103D8000C35CDB4F88830091590610E0C7018E5B4E
:103D90009F4F0E94EB0AF801ED5FFB4F882319F05B
:103DA0008081886002C08081877F808380915906EE
:103DB000C82FD0E0C7018C5B9F4F0E94EB0AC95C03
:103DC000DB4F888380915906C82FD0E0C7018A5BFA
:103DD0009F4F0E94EB0A90E00E94951CC75CDB4F4E
:103DE00088830091590610E0C701805B9F4F0E94B5
:103DF000EB0AF801ED5FFB4F882319F080818062A8
:103E000002C080818F7D808380915906C82FD0E0C9
:103E1000C7018E5A9F4F0E94EB0AC15CDB4F88831B
:103E200080915906C82FD0E0C7018C5A9F4F0E943D
:103E3000EB0A90E00E94951CCF5BDB4F88830091DA
:103E4000590610E0C7018A5A9F4F0E94EB0AF801F9
:103E5000ED5FFB4F882319F08081806402C0808170
:103E60008F7B808380915906C82FD0E0C701885A84
:103E70009F4F0E94EB0ACD5BDB4F888380915906F0
:103E8000C82FD0E0C701865A9F4F0E94EB0A90E0EE
:103E90000E94951CCB5BDB4F88830091590610E094
:103EA000C70182569F4F0E94EB0AF801ED5FFB4F5E
:103EB000882319F08081806802C080818F77808399
:103EC00080915906C82FD0E0C70180569F4F0E94AD
:103ED000EB0AC95BDB4F888380915906C82FD0E07D
:103EE000C7018E559F4F0E94EB0A90E00E94951CDF
:103EF000C75BDB4F88830091590610E0C7018E59DC
:103F00009F4F0E94EB0AF801EB5FFB4F882319F0EB
:103F10008081816002C080818E7F8083809159067C
:103F2000C82FD0E0C7018C599F4F0E94EB0AC55B98
:103F3000DB4F888380915906C82FD0E0C7018A598A
:103F40009F4F0E94EB0A90E00E94951CC35BDB4FE1
:103F500088830091590610E0C70182599F4F0E9443
:103F6000EB0AF801EB5FFB4F882319F08081846036
:103F700002C080818B7F808380915906C82FD0E05A
:103F8000C70180599F4F0E94EB0AC15BDB4F8883BA
:103F900080915906C82FD0E0C7018E589F4F0E94CC
:103FA000EB0A90E00E94951CCF5ADB4F888300916A
:103FB000590610E0C70184579F4F0E94EB0AF80191
:103FC000EB5FFB4F882319F08081806802C08081FD
:103FD0008F77808380915906C82FD0E0C701825720
:103FE0009F4F0E94EB0ACD5ADB4F88838091590680
:103FF000C82FD0E0C70180579F4F0E94EB0A90E086
:104000000E94951CCB5ADB4F88830091590610E023
:10401000C7018E569F4F0E94EB0AF801EB5FFB4FE2
:10402000882319F08081826002C080818D7F808327
:1040300080915906C82FD0E0C7018C569F4F0E942F
:10404000EB0AC55ADB4F888380915906C82FD0E010
:10405000C7018A569F4F0E94EB0A90E00E94951C70
:10406000C35ADB4F88830091590610E0C7018C5872
:104070009F4F0E94EB0AF801EB5FFB4F882319F07A
:104080008081886002C08081877F8083809159060B
:10409000C82FD0E0C7018A589F4F0E94EB0AC95A27
:1040A000DB4F888380915906C82FD0E0C70188581C
:1040B0009F4F0E94EB0A90E00E94951CC75ADB4F6D
:1040C00088830091590610E0C70186589F4F0E94CF
:1040D000EB0AF801EB5FFB4F882319F080818061C8
:1040E00002C080818F7E808380915906C82FD0E0E6
:1040F000C70184589F4F0E94EB0AC15ADB4F888347
:1041000080915906C82FD0E0C70182589F4F0E9466
:10411000EB0A90E00E94951CCF59DB4F88830091F9
:10412000590610E0C70180589F4F0E94EB0AF80122
:10413000EB5FFB4F882319F08081806202C0808191
:104140008F7D808380915906C82FD0E0C7018E579C
:104150009F4F0E94EB0ACD59DB4F8883809159060F
:10416000C82FD0E0C7018C579F4F0E94EB0A90E008
:104170000E94951CCB59DB4F88830091590610E0B3
:10418000C7018A579F4F0E94EB0AF801EB5FFB4F74
:10419000882319F08081806402C080818F7B8083B6
:1041A00080915906C82FD0E0C70188579F4F0E94C1
:1041B000EB0AC959DB4F888380915906C82FD0E09C
:1041C000C70186579F4F0E94EB0A90E00E94951C02
:1041D000C759DB4F88830091590610E0C7018C5501
:1041E0009F4F0E94EB0AF801E95FFB4F882319F00B
:1041F0008081816002C080818E7F8083809159069A
:10420000C82FD0E0C7018A559F4F0E94EB0AC559BD
:10421000DB4F888380915906C82FD0E0C7018855AD
:104220009F4F0E94EB0A90E00E94951CC359DB4F00
:1042300088830091590610E0C70180559F4F0E9466
:10424000EB0AF801E95FFB4F882319F08081846055
:1042500002C080818B7F808380915906C82FD0E077
:10426000C7018E549F4F0E94EB0AC159DB4F8883D0
:1042700080915906C82FD0E0C7018C549F4F0E94EF
:10428000EB0A90E00E94951CCF58DB4F8883009189
:10429000590610E0C7018A549F4F0E94EB0AF801AB
:1042A000E95FFB4F882319F08081886002C080811C
:1042B000877F808380915906C82FD0E0C70188543A
:1042C0009F4F0E94EB0ACD58DB4F8883809159069F
:1042D000C82FD0E0C70186549F4F0E94EB0A90E0A0
:1042E0000E94951CCB58DB4F88830091590610E043
:1042F000C70184549F4F0E94EB0AF801E95FFB4F0E
:10430000882319F08081806102C080818F7E808344
:1043100080915906C82FD0E0C70182549F4F0E9458
:10432000EB0AC958DB4F888380915906C82FD0E02B
:10433000C70180549F4F0E94EB0A90E00E94951C99
:10434000C758DB4F88830091590610E0C701845A93
:104350009F4F0E94EB0AF801E95FFB4F882319F099
:104360008081806402C080818F7B80838091590628
:10437000C82FD0E0C701825A9F4F0E94EB0AC55850
:10438000DB4F888380915906C82FD0E0C701805A3F
:104390009F4F0E94EB0A90E00E94951CC358DB4F90
:1043A00088830091590610E0C70180529F4F0E94F8
:1043B000EB0AF801E75FFB4F882319F080818460E6
:1043C00002C080818B7F808380915906C82FD0E006
:1043D000C7018E519F4F0E94EB0AC158DB4F888363
:1043E00080915906C82FD0E0C7018C519F4F0E9481
:1043F000EB0A90E00E94951CCF57DB4F8883009119
:10440000590610E0C7018C529F4F0E94EB0AF80139
:10441000E75FFB4F882319F08081826002C08081B2
:104420008D7F808380915906C82FD0E0C7018A52C2
:104430009F4F0E94EB0ACD57DB4F8883809159062E
:10444000C82FD0E0C70188529F4F0E94EB0A90E02E
:104450000E94951CCB57DB4F8883DF91CF911F9132
:104460000F91FF90EF9008954F925F927F928F92FD
:104470009F92AF92BF92CF92DF92EF92FF920F93F3
:104480001F93DF93CF93CDB7DEB7C854D0400FB69C
:10449000F894DEBF0FBECDBF04EA14E0C8010E944D
:1044A0009405C80166E049E00E946F04C8010E94BB
:1044B000470500D000D0EDB7FEB7128301838FEF20
:1044C00091E0948383830E94BE290F900F900F90F8
:1044D0000F90C8010E942B0500D000D007E814E01F
:1044E000EDB7FEB7128301838FEE91E0948383834F
:1044F0000E94BE2954EE452E51E0552EEE24FF2495
:10450000CC24DD240F900F900F900F90702E012F70
:1045100049E0A42EB12CAC0EBD1E4E010894811CA6
:10452000911C87E894E00E94722A982F8D3031F018
:104530008D30DCF180538230C0F530C01830A1F5E9
:104540009981892F8053823078F5913311F490E866
:1045500001C090E08A81813309F4905C8B818133C2
:1045600009F4905E8C81813309F4905F8D818133F1
:1045700009F4985F8E81813309F49C5F8F818133C8
:1045800009F49E5F8885813309F49F5FF501EE0D84
:10459000FF1D90830894E11CF11C06C0F401E10F9B
:1045A000F11D90831F5F01C010E0F0E4EF16F104ED
:1045B000C9F484EA94E0B601A5010E947F0408943E
:1045C000C11CD11C00D000D0EDB7FEB771820283B0
:1045D000548243820E94BE29EE24FF240F900F9044
:1045E0000F900F90FFEFCF16D10409F00CF499CF84
:1045F000C85BDF4F0FB6F894DEBF0FBECDBFCF91C3
:10460000DF911F910F91FF90EF90DF90CF90BF90BF
:10461000AF909F908F907F905F904F900895DF9222
:10462000EF92FF920F931F93DF93CF93CDB7DEB737
:104630002A970FB6F894DEBF0FBECDBF73E0E72E0A
:10464000F12CEC0EFD1E63E0D62E21C40E946831D1
:1046500060527E4480409040C8F40E94683169589E
:1046600073418040904090F01A3011F01D3031F4C9
:10467000809123068F5F8093230602C01092230649
:1046800080912306833011F40E943422812F69E146
:1046900075E00E94F106882311F400E0F2C38091D6
:1046A0001D0590911E05A0911F05B0912005863E25
:1046B00046EA940746E2A4074DE7B40709F4A0C20E
:1046C000873E56EA950756E2A5075DE7B50708F06D
:1046D000F8C08832EEE59E07E2EDAE07E4E2BE07E1
:1046E00009F439C28932FEE59F07F2EDAF07F4E223
:1046F000BF0708F073C080352FED92072DEEA2079B
:1047000028E1B20709F479C381353FED93073DEE07
:10471000A30738E1B30788F584304AE9940747EDE9
:10472000A4074EE0B40709F416C285305AE995078C
:1047300057EDA5075EE0B50780F48E3FEBEC9E07D2
:10474000E7ECAE07E9E0BE0709F482C386519A4A56
:10475000A743BB4009F08BC3FEC1823923EA92070D
:104760002CEEA20724E1B20709F4F5C188599C4256
:10477000AA41B64109F07BC3F7C184344BED9407DD
:1047800040E7A4074DE1B40709F462C385345BED4B
:10479000950750E7A5075DE1B50780F48E3CE8E496
:1047A0009E07E7E5AE07EAE1BE0709F429C2845790
:1047B0009B4EAA47BB4109F05AC3CDC1823D22ECB2
:1047C000920722E8A2072EE1B20709F4CDC18C5A64
:1047D0009A4CA64EB04209F04AC33AC3883546EB1C
:1047E00094074DEFA4074AE4B40709F4E8C28935F9
:1047F00056EB95075DEFA5075AE4B50788F5863EA9
:10480000E5ED9E07EAEDAE07E3E3BE0709F451C10B
:10481000873EF5ED9F07FAEDAF07F3E3BF0780F49E
:104820008E3729EA92072BE5A20726E2B20709F4A0
:104830009BC182559342A649B64209F018C36FC284
:10484000883F4CEA94074EEEA40744E3B40709F40A
:10485000FFC2865A9E40A241B84409F008C398C2DC
:104860008036EBED9E07EBE3AE07EEE6BE0709F4FC
:1048700072C18136FBED9F07FBE3AF07FEE6BF0782
:1048800080F4823E25E592072CE9A20726E6B207CE
:1048900009F4A5C28C5E9943A647BB4609F0E7C25E
:1048A000D7C28A3B47EC940741E2A40744E7B40728
:1048B00009F4FFC08A57974CA94DBB4709F0D7C2EE
:1048C000C7C28C36E8E69E07E3E4AE07E2ECBE071B
:1048D00009F406C28D36F8E69F07F3E4AF07F2EC61
:1048E000BF0708F073C08A3726EF920721EFA207AF
:1048F0002DE9B20709F484C18B3736EF930731EF06
:10490000A3073DE9B30788F58C3845E8940747EAE3
:10491000A40748E9B40709F473C18D3855E8950731
:1049200057EAA50758E9B50780F48634E3E09E0707
:10493000E2ECAE07E5E8BE0709F491C282559A4E53
:10494000A048BA4809F093C206C18A362EE29207FF
:1049500022E6A20729E9B20709F41AC28E5792414A
:10496000AA46BB4909F083C2F6C08A3847EF9407CC
:1049700047ECA40748EBB40709F4F6C08B3857EFAF
:10498000950757ECA50758EBB50780F48E3FE6EB8B
:104990009E07E9E2AE07E5EABE0709F431C180529D
:1049A0009E44A94AB14B09F062C219C2843A20E080
:1049B00092072BE9A2072AEBB20709F449C28A5BE6
:1049C0009448A542BE4B09F052C209C2843649ED53
:1049D000940740EEA40747EDB40709F46AC0853692
:1049E00059ED950750EEA50757EDB50788F58435C5
:1049F000EDE29E07EFEFAE07E5ECBE0709F4ABC0B2
:104A00008535FDE29F07FFEFAF07F5ECBF0780F4A8
:104A1000803824E7920720E1A20724ECB20709F4CA
:104A2000A3C086589B43A04AB44C09F020C2D7C10A
:104A300088324FE9940740E0A40747ECB40709F433
:104A40005FC186599543A840B24D09F010C267C1B5
:104A50008E34EDE59E07EEE3AE07E3EEBE0709F404
:104A60007AC08F34FDE59F07FEE3AF07F3EEBF0783
:104A700080F4843727E3920724EDA2072EEDB207D6
:104A800009F4ADC1865B9342A34AB24E09F0EFC16F
:104A9000B7C0823940E7940746E8A4074BEFB40754
:104AA00009F4D6C1825F9D4EA442BD4F09F0DFC11B
:104AB0009FC10E9468316093C8047093C9048093B9
:104AC000CA049093CB04D092C70489E195E060E1D9
:104AD00070E00E94C5080E9470347093CD0460930A
:104AE000CC0489E195E064E170E00E94C5080E9471
:104AF00070347093CF046093CE0489E195E068E14F
:104B000070E00E94C5080E9470348B017093D1043C
:104B10006093D0046091D2047091D3048091D40446
:104B20009091D50420E030E040E050E00E94013454
:104B3000882379F4B801882777FD8095982F0E9403
:104B4000A3346093D6047093D7048093D8049093D1
:104B5000D90401E08DC1809123058093DA0480910E
:104B600024058093DB0483C189E195E060E070E077
:104B70000E94C50820E030E048EC52E40E94D6359F
:104B80000E9470347093DD046093DC04693C71050D
:104B900020F01092DD041092DC0480913D0590918C
:104BA0003E059093DF048093DE0480913F05909151
:104BB00040059093E1048093E00480914305909137
:104BC00044059093A4028093A3028091470590919D
:104BD00048059093A6028093A50280914905909183
:104BE0004A059093A8028093A70280914B0590916B
:104BF0004C059A8389839093AA028093A90237C1B6
:104C000060912305709124058091250590912605DA
:104C10000E94A33420E836E948E15BE40E940834AE
:104C20006093D2047093D3048093D4049093D504FA
:104C300060912705709128058091290590912A059A
:104C4000D7016C9311967C93119712968C931297BF
:104C500013969C930E94A33420E836E948E15BE474
:104C60000E9408346093E2047093E3048093E404A8
:104C70009093E504809148058093E6048091470570
:104C800084300CF083E08093E70489E195E060E1F3
:104C900070E00E94C5086093D6047093D704809397
:104CA000D8049093D90489E195E068E070E00E940F
:104CB000C5086093E8047093E9048093EA04909334
:104CC000EB0489E195E064E170E00E94C50860931F
:104CD000EC047093ED048093EE049093EF04C7C04E
:104CE00089E195E068E070E00E94C5089058609303
:104CF000F0047093F1048093F2049093F304B7C02E
:104D000089E195E060E070E00E94C5086093F404DA
:104D10007093F5048093F6049093F704A8C089E19A
:104D200095E060E070E00E94C5086093F80470931D
:104D3000F9048093FA049093FB0489E195E064E020
:104D400070E00E94C50820E030E048EC52E40E9488
:104D5000D6350E9470347093FD046093FC0489E1A1
:104D600095E064E170E00E94C5080E947034709381
:104D7000FF046093FE0489E195E068E170E00E9421
:104D8000C5080E94703470930105609300056FC0E0
:104D900089E195E064E070E00E94C5080E947034EB
:104DA000882777FD8095982F0E94A3346093020591
:104DB00070930305809304059093050558C089E11D
:104DC00095E068E070E00E94C5080E94703470951C
:104DD00061957F4F709307056093060548C08091E9
:104DE00083058093080580918405809309053FC061
:104DF0008091230580930A053AC089E195E060E03F
:104E000070E00E94C50860930B0570930C058093B9
:104E10000D0590930E0589E195E064E070E00E9435
:104E2000C50860930F05709310058093110590934A
:104E3000120589E195E068E070E00E94C508609382
:104E400013057093140580931505909316050FC0F4
:104E500080912F05809317058091340506C08091BD
:104E6000300580931705809135058093180500E083
:104E700080911A05823229F489E195E063E20E946B
:104E8000DD098EEB90E00E94CF31002331F587E8F9
:104E900094E00E94422A18161906F4F487E894E078
:104EA0000E94722A182F8091C704882309F0EECB44
:104EB000CDCB1092C70401E0802F90E02A960FB668
:104EC000F894DEBF0FBECDBFCF91DF911F910F9140
:104ED000FF90EF90DF90089500E02091C80430919A
:104EE000C9044091CA045091CB04205F384D4F4F04
:104EF0005F4F2F83388749875A870E9468312F81F7
:104F0000388549855A85261737074807590788F293
:104F1000D3CF1F93CF93DF9385E090E06CE070E0F8
:104F20000E940E1668EE73E080E090E00E947631F9
:104F300087E894E00E94BF2AC0E0D0E010E0CE01F4
:104F40006DE171E00E941037892BA9F41F5E84EA9D
:104F500094E0612F4CE00E946F0484EA94E00E9488
:104F6000470584EA94E06EEE0E94770584EA94E0B7
:104F70000E942B05105161E070E080E090E00E94FB
:104F80007631219687E0C13DD807C9F6DF91CF91F0
:104F90001F91089586E061E00E94AD3208950F935D
:104FA0001F9386E061E00E946E3207E814E0C801BA
:104FB00040E051EE60E070E00E94E0291093A2060C
:104FC0000093A1060E94CA2784EA94E00E94CD05BE
:104FD0000E948C1C64EF71E080E090E00E947631CA
:104FE00083EF93E00E94EB0A813011F00E94FC0CE9
:104FF0000E945C0A1092590607C00E94AA1C809168
:1050000059068F5F80935906809159068230A8F324
:10501000109259060E94892786EB94E06EE979E2A6
:1050200024E630E040E050E000E00E94933084EA63
:1050300094E00E94940586EB94E00E94F9301F9161
:105040000F9108952F923F924F925F926F927F92AD
:105050008F929F92AF92BF92CF92DF92EF92FF9288
:105060000F931F93DF93CF9300D000D0CDB7DEB75F
:1050700080915506882309F4E1C0E0907A06F0900B
:105080007B0600917C0610917D06C801B7019F77D1
:1050900025E33AEF4EE85CE30E94D6350E940534E2
:1050A00069837A838B839C83C801B7012091D204E2
:1050B0003091D3044091D4045091D5040E943A33E6
:1050C0001B012C019F7720EC3BE649ED57E40E9441
:1050D000D6355B016C0160917E0670917F068091F0
:1050E0008006909181062091E2043091E304409182
:1050F000E4045091E5040E943A333B014C019F7750
:1051000020EC3BE649ED57E40E94D63529813A81EF
:105110004B815C810E94D6357B018C01C601B501B3
:10512000A60195010E94D6355B016C01C801B7014B
:10513000A80197010E94D6359B01AC01C601B501BB
:105140000E943B330E945D360E9470346093480693
:105150007093490680934A0690934B0660E070E096
:1051600080E89FE329813A814B815C810E94083469
:105170009B01AC01C201B1010E94D63597FA90940F
:1051800097F89094A40193010E94AE3320EE3EE282
:1051900045E652E40E94D63520E030E044EB52E48C
:1051A0000E943B330E9470349B01AC0197FF04C006
:1051B00028593E4F4F4F5F4FCA01B901645B7040A1
:1051C0008040904097FF06C0CA01B9016C547F4FE0
:1051D0008F4F9F4F0E94A3342091D6043091D70463
:1051E0004091D8045091D9040E943A330E947034FF
:1051F00097FF04C068597E4F8F4F9F4F0E94A33482
:1052000020E030E044EB53E40E94083420E030E03A
:1052100040E851E40E94D6350E94393620E030E063
:1052200040E85FE30E943B330E9475346093470679
:10523000613108F46CC01092470669C08091E704A0
:10524000823008F464C08091E604853008F45FC0C1
:10525000A09082068DE18A1508F459C0E090E80418
:10526000F090E9040091EA041091EB046091830648
:10527000709184068091850690918606A801970119
:105280000E943A339F7720E030E040E05FE30E94E5
:10529000CB3518165CF410928206E0928306F092E9
:1052A0008406009385061093860631C08A2D8F5F91
:1052B000809382068E3159F58091D2049091D30467
:1052C000A091D404B091D50480937A0690937B0684
:1052D000A0937C06B0937D068091E2049091E30454
:1052E000A091E404B091E50480937E0690937F063C
:1052F000A0938006B0938106E0928706F09288061C
:105300000093890610938A0681E0809355060F90DA
:105310000F900F900F90CF91DF911F910F91FF9001
:10532000EF90DF90CF90BF90AF909F908F907F9045
:105330006F905F904F903F902F90089580910A0555
:105340008093AB021092AC020E944E080E94F10AB8
:1053500084EA94E00E9422280E945B1A08950E9429
:105360000F23892B19F00E949E29089586EB94E063
:105370000E94E13008958FEF9FE70895DF93CF9368
:10538000CDB7DEB7FE0139968D819E8161E04F81F8
:1053900058859F010E945F2CCF91DF910895DF9384
:1053A000CF93CDB7DEB7FE0139968D819E8160E047
:1053B0004F8158859F010E945F2CCF91DF91089506
:1053C0000F931F93DC01ED91FC910288F389E02D8E
:1053D00020E030E000E010E009951F910F91089562
:1053E0008F92AF92CF92EF92FF920F931F93DF9322
:1053F000CF93CDB7DEB7FC011382128288EE93E023
:10540000A0E0B0E084839583A683B78389EE93E020
:10541000918380835587448737872687118B008B3C
:10542000F38AE28AC48AA58A868A70E0CB0123E0E7
:10543000880F991F2A95E1F79C012157394F308F2A
:10544000278B8956994F928F818F81E090E002C01F
:10545000880F991F6A95E2F720919F06282B2093C9
:105460009F06CF0140E051EE60E070E00E94E0292D
:10547000CF91DF911F910F91FF90EF90CF90AF9060
:105480008F900895FC01838D882319F42FEF3FEF4F
:105490000DC00788F08DE02D2081318182819381BC
:1054A000281B390B8481958128233923C90108954C
:1054B000FC01838D882319F42FEF3FEF11C0018C7D
:1054C000F28DE02D2081318182819381281B390B5F
:1054D0002095309584819581282339232F5F3F4F74
:1054E000C9010895FC01838D882361F0A789B08DDF
:1054F0002D913C91119712968D919C91139728179D
:10550000390721F44FEF5FEFCA01089512968D918C
:105510009C9113971696ED91FC911797E80FF91F40
:10552000408112968D919C911397019614962D911E
:105530003C9115978223932313969C938E931297F5
:1055400050E0E2CFFC01838D882351F00788F08D75
:10555000E02D20813181828193812817390721F440
:105560002FEF3FEFC9010895828193810680F78173
:10557000E02DE80FF91F8081282F30E0F3CFDC0108
:105580005796ED91FC915897828193819183808306
:105590005996ED91FC915A978081918193838283F2
:1055A0000895DC015B968C915B978823A9F159964D
:1055B000ED91FC915A97208131812F5F3F4F84817B
:1055C0009581282339235C968C915C97882329F058
:1055D0008281938128173907F9F0828193812817F6
:1055E0003907D9F3808191810680F781E02DE80F9A
:1055F000F91F60835996ED91FC915A97318320836E
:105600005296ED91FC915397808156969C91892BEF
:10561000808321E030E002C020E030E0C90108953D
:10562000CF93DF93EC011B821A828A819B8199833D
:1056300088831D821C828E819F81009721F00E94A9
:10564000C1031F821E82DF91CF9108950F931F9394
:105650008C01DC015296ED91FC9153972081569676
:105660008C91569755969C915597892B80958223BE
:10567000808357968D919C9158970E94102BF8012A
:10568000818D928D0E94102BD8015B961C921F91E8
:105690000F9108950F931F93CF93DF938C01FC011B
:1056A00013821282828193819183808341E0A1E001
:1056B000B0E001C04F5FFD01042E02C0EE0FFF1FDE
:1056C0000A94E2F79B0182E06130780710F020E055
:1056D00032E0E217F30770F3C1E0D0E002C0CC0F74
:1056E000DD1F4A95E2F72197F801268137812115C0
:1056F000310541F0848195818C179D0789F0C9019E
:105700000E94C103F801D583C483CE0101960E9493
:1057100017039C01F8019783868380E0232B09F00F
:1057200081E0DF91CF911F910F910895AF92BF92C9
:10573000CF92DF92EF92FF920F931F93CF93DF935D
:105740007C015A016B01E901DC015B968C915B974E
:105750008823F1F02115310539F45796ED91FC912C
:105760005897C481D58121960115110549F4D701B7
:105770005996ED91FC915A97048115810F5F1F4F47
:10578000D701ED91FC910088F189E02DC7010995C1
:10579000F7018789908D209711F4C0E8D0E0BE0111
:1057A0000E944A2B882381F0D70159968D919C91B4
:1057B0005A970115110511F400E110E0B8010E949B
:1057C0004A2B882309F04DC0D701ED91FC91008848
:1057D000F189E02DC701099567C0D7015096ED9179
:1057E000FC915197B0E0AB16B1EEBB06B0E0CB0632
:1057F000B0E0DB0609F454C081E090E0D701549694
:105800000C9002C0880F991F0A94E2F7808360E031
:1058100079E08DE390E0A60195010E944537215083
:10582000304040405040CA01B90122E030E040E041
:1058300050E00E944537D7011C96ED91FC911D97D1
:1058400030831E96ED91FC911F972083D7015296CD
:10585000ED91FC915397808155969C91892B808383
:1058600023C0D7015996ED91FC915A971382128269
:1058700082819381918380835796ED91FC91589713
:1058800013821282828193819183808381E05B966F
:105890008C931A141B041C041D040CF49ECFD6CF49
:1058A000108220E130E0C7CFDF91CF911F910F919F
:1058B000FF90EF90DF90CF90BF90AF9008952F9220
:1058C0003F924F925F926F927F928F929F92AF9290
:1058D000BF92CF92DF92EF92FF920F931F93DF93CD
:1058E000CF93CDB7DEB764970FB6F894DEBF0FBE87
:1058F000CDBF3C01688B5A8B498B69011C01AE01FD
:105900004F5F5F4F5C8B4B8BE989FA89488940FD7B
:10591000659140FF6191FA8BE98B662309F4D7C347
:10592000653249F440FD859140FF8191FA8BE98B06
:105930008532B1F40CC06A3051F4D301ED91FC9181
:105940000190F081E02DC1016DE009956AE0D3017D
:10595000ED91FC910190F081E02DC1010995D4CF2A
:10596000982F10E0882499241032B0F49B3269F00B
:105970009C3228F4903251F0933271F40BC09D3276
:1059800039F0903349F4116028C01260146025C0CA
:10599000186023C0106121C017FD2BC0892F8053D0
:1059A0008A3078F416FF06C0BAE09B9E902C112432
:1059B000980E13C0EAE08E9E802C1124880E10628F
:1059C0000CC09E3221F416FD82C3106406C09C36C2
:1059D00011F4106802C0983661F4E989FA8948899F
:1059E00040FD959140FF9191FA8BE98B992309F045
:1059F000BBCF892F8554833020F4812F8061905E46
:105A000007C0892F8556833008F0E6C1812F8F7E2D
:105A100086FD02C076E0972E6FE3F62EF8229536CB
:105A200019F450E4F52A07C0963619F480E8F82AEC
:105A300002C091109A94F7FE0BC09BE3991520F4D5
:105A400027E05CE3B52E0DC0B92CB39427E009C064
:105A5000A7E0A91520F447E0942E27E001C0292DE6
:105A6000BB24F6013496FD87EC87D6016D917D91BC
:105A70008D919C91AE014F5F5F4F0B2D0E943F02B5
:105A80006C010981E02FF0E0FF87EE8700FF05C081
:105A9000FE85F3FD02C01DE209C0F1FE02C01BE25B
:105AA00005C0F2FC02C010E001C010E28E859F85A7
:105AB0008C709070892B09F444C0112311F483E099
:105AC00001C084E0881510F088240EC0881AF3FC09
:105AD0000BC0D301ED91FC910190F081E02DC1014B
:105AE00060E209958A94A9F7112349F0D301ED9159
:105AF000FC910190F081E02DC101612F0995BE85D7
:105B0000B3FF03C008E013E012C00CE013E00FC0C5
:105B1000E114F10409F06052D301ED91FC91019080
:105B2000F081E02DC10109950F5F1F4F05C0EF2CDB
:105B3000FF24B0E1EB22FF24F8016491662341F7D2
:105B400048C1F7FE13C0BC0CFE85F4FF04C08A8177
:105B5000813309F4BA941B141CF0BB24B3942DC0F8
:105B600048E04B1550F538E0B32E27C0F6FC25C0B1
:105B7000892D90E08C159D054CF05CEFC5165FEF0C
:105B8000D50624F080E8F82A01C09A94992049F0BB
:105B9000E2E0F0E0EC0FFD1FE90DF11D80818033A4
:105BA000A1F3F7FE0AC0B92CB394892D90E0C81672
:105BB000D90614F0992401C09C18F7FC03C025E015
:105BC00030E009C01C141D041CF021E030E003C0CB
:105BD00096012F5F3F4F112311F02F5F3F4F992008
:105BE00029F0892D90E00196280F391F882D90E02B
:105BF0002817390714F0882401C0821A4F2C552425
:105C0000C20189709070892B59F00CC0D301ED91BD
:105C1000FC910190F081E02DC10160E209958A9428
:105C20008820A1F7112349F0D301ED91FC91019057
:105C3000F081E02DC101612F099543FE0BC00CC01E
:105C4000D301ED91FC910190F081E02DC10160E361
:105C500009958A948820A1F7F7FE51C08601D7FEE6
:105C600002C000E010E076010894E11CF11CE01A8B
:105C7000F10AE1E0F0E0EC0FFD1FEE0EFF1E260141
:105C80004B185108892D90E0AA24BB24A81AB90A00
:105C9000FFEF0F3F1F0749F4D301ED91FC910190F5
:105CA000F081E02DC1016EE20995C016D10634F0F5
:105CB000401651061CF4F701608101C060E30150F9
:105CC00010400894E11CF11C0A151B054CF0D3018F
:105CD000ED91FC910190F081E02DC1010995D8CFA3
:105CE0000C151D0541F48A81863320F4853319F49F
:105CF000BE85B4FF61E3D301ED91FC9165C06A817B
:105D0000613309F00F7ED301ED91FC910190F08198
:105D1000E02DC10109959920E1F0D301ED91FC91AD
:105D20000190F081E02DC1016EE2099512E0E1E001
:105D3000F0E0EC0FFD1FE10FF11D60811F5FD3014B
:105D4000ED91FC910190F081E02DC10109959A94AB
:105D500071F7D301ED91FC910190F081E02D44FCAD
:105D600002C065E601C065E4C1010995D7FC05C024
:105D7000C114D10441F404FF06C0D094C194D108E9
:105D8000D3946DE201C06BE2D301ED91FC910190DF
:105D9000F081E02DC101099560E305C06F5FE6EF7A
:105DA000FFEFCE0EDF1EFAE0CF16D104BCF7D30111
:105DB000ED91FC910190F081E02DC1010995D30195
:105DC000ED91FC916C2D605D0190F081E02DC101A1
:105DD0000995CC84DD8478C1933631F0933799F0FE
:105DE000933509F061C023C0F601808189835E018B
:105DF0000894A11CB11C42E050E0C40ED51E21E065
:105E0000E22EF12C12C0D601AD90BC9016FD03C05D
:105E10006FEF7FEF02C0692D70E0E2E0F0E0CE0EA0
:105E2000DF1EC5010E9424047C011F7713C0D60128
:105E3000AD90BC9016FD03C06FEF7FEF02C0692DDF
:105E400070E0E2E0F0E0CE0EDF1EC5010E94190412
:105E50007C01106813FF0BC023C0D301ED91FC91AE
:105E60000190F081E02DC10160E209958A94882DAE
:105E700090E0E816F90688F313C0F50117FD659167
:105E800017FF61915F01D301ED91FC910190F081C9
:105E9000E02DC101099581108A940894E108F10868
:105EA000E114F10451F710C1943611F0993699F5C7
:105EB00017FF0AC0F601208131814281538184E0BD
:105EC00090E0C80ED91E0CC0D6018D919C919C010A
:105ED000442737FD4095542FE2E0F0E0CE0EDF1E60
:105EE0009FE6F92EF12257FF09C050954095309555
:105EF00021953F4F4F4F5F4FF0E8FF2ACA01B9018C
:105F0000AE014F5F5F4F2AE030E00E94E101E82ED2
:105F10004B89E41A41C0953721F41F7E2AE030E016
:105F20001CC0197F9F3661F0903720F4983509F036
:105F3000CEC00FC0903739F0983709F0C8C004C000
:105F400028E030E00AC0106114FD146020E130E068
:105F500004C014FD166020E132E017FF08C0D6012E
:105F60006D917D918D919C91E4E0F0E008C0D601A7
:105F70008D919C91BC0180E090E0E2E0F0E0CE0EDB
:105F8000DF1EAE014F5F5F4F0E94E101E82EFB89EB
:105F9000EF1A8FE7F82EF122F6FE0BC04EEFF42237
:105FA000E91438F4F4FE07C0F2FC05C05FEEF522F8
:105FB00002C01E2D01C0192DF4FE0DC0FE01EE0D14
:105FC000F11D8081803319F489EEF82208C01F5F2B
:105FD000F2FE05C003C08F2D867809F01F5F0F2DDC
:105FE000F3FC18C0F0FE13C0181510F09E2C0FC063
:105FF0009E2C980C911A182D0AC0D301ED91FC919A
:106000000190F081E02DC10160E209951F5F181534
:10601000A0F304C0181510F4811A01C0882404FFED
:1060200017C0D301ED91FC910190F081E02DC101E9
:1060300060E3099502FF29C0D301ED91FC91019025
:10604000F081E02D01FD02C068E712C068E510C0D4
:10605000802F8678D1F001FF02C06BE201C060E2C0
:10606000F7FC6DE2D301ED91FC910190F081E02D00
:10607000C10109950AC0D301ED91FC910190F08115
:10608000E02DC10160E309959A94E914A0F3EA9424
:10609000D301ED91FC91A1E0B0E0AC0FBD1FAE0DBE
:1060A000B11D0190F081E02DC1016C910995EE20A8
:1060B00071F70AC0D301ED91FC910190F081E02DC0
:1060C000C10160E209958A948820A1F71DCC6496ED
:1060D0000FB6F894DEBF0FBECDBFCF91DF911F91F9
:1060E0000F91FF90EF90DF90CF90BF90AF909F9077
:1060F0008F907F906F905F904F903F902F9008957A
:10610000F999FECF72BD61BDF89A80B50895F999ED
:10611000FECF1FBA72BD61BD40BD0FB6F894FA9AAA
:10612000F99A0FBE08950F93FC016115710511F4E2
:1061300080E011C021833283438354837287618757
:106140000170000F000F000F8081877F802B82601D
:106150008B7F808381E00F910895CF93DF93EC01D3
:106160000E9468319B01AC018D819E81AF81B88511
:10617000281739074A075B0728F4888184FD02C085
:1061800060E00DC089819A81AB81BC81820F931F31
:10619000A41FB51F8D839E83AF83B88761E022273C
:1061A00057FD2395332744275527922F91709295B9
:1061B000907F88818F7E892B8883862FDF91CF9176
:1061C0000895CF93DF93EC01888182FF0FC0CE0149
:1061D0000E94AD30882351F0E985FA85309709F0A7
:1061E0000995888183FF02C08B7F8883DF91CF91DF
:1061F0000895CF93DF93EC0189859A85892BE1F08F
:1062000089819A81AB81BC810097A105B105A1F07C
:106210000E94683129813A814B815C81260F371FAA
:10622000481F591F2D833E834F8358878881846080
:106230008F7E888381E001C080E0DF91CF91089557
:106240001F920F920FB60F9211242F933F938F93AB
:106250009F93AF93BF938091A7069091A806A091BA
:10626000A906B091AA063091AB060196A11DB11DF9
:10627000232F2D5F2D3720F02D570196A11DB11D25
:106280002093AB068093A7069093A806A093A90637
:10629000B093AA068091A3069091A406A091A506AA
:1062A000B091A6060196A11DB11D8093A3069093FF
:1062B000A406A093A506B093A606BF91AF919F91A7
:1062C0008F913F912F910F900FBE0F901F901895B7
:1062D0008FB7F8942091A7063091A8064091A9069F
:1062E0005091AA068FBFB901CA0108959B01AC0164
:1062F0007FB7F8948091A3069091A406A091A5067B
:10630000B091A60666B5A89B05C06F3F19F001962F
:10631000A11DB11D7FBFBA2FA92F982F8827860FE7
:10632000911DA11DB11D62E0880F991FAA1FBB1FFF
:106330006A95D1F7BC012DC0FFB7F8948091A306F0
:106340009091A406A091A506B091A606E6B5A89BDB
:1063500005C0EF3F19F00196A11DB11DFFBFBA2F77
:10636000A92F982F88278E0F911DA11DB11DE2E046
:10637000880F991FAA1FBB1FEA95D1F7861B970BA1
:10638000885E9340C8F221503040404050406851F0
:106390007C4F211531054105510571F6089501978E
:1063A00039F0880F991F880F991F02970197F1F70D
:1063B0000895789484B5826084BD84B5816084BD7D
:1063C00085B5826085BD85B5816085BDEEE6F0E06E
:1063D000808181608083E1E8F0E0108280818260CA
:1063E0008083808181608083E0E8F0E0808181604B
:1063F0008083E1EBF0E0808184608083E0EBF0E07B
:10640000808181608083EAE7F0E08081846080831E
:1064100080818260808380818160808380818068C8
:1064200080831092C10008951F920F920FB60F92B1
:1064300011242F933F934F935F936F937F938F9389
:106440009F93AF93BF93EF93FF938091AC0690918E
:10645000AD06892B29F0E091AC06F091AD060995C7
:10646000FF91EF91BF91AF919F918F917F916F912C
:106470005F914F913F912F910F900FBE0F901F9002
:1064800018951F920F920FB60F9211242F933F93DE
:106490004F935F936F937F938F939F93AF93BF932C
:1064A000EF93FF938091AE069091AF06892B29F070
:1064B000E091AE06F091AF060995FF91EF91BF9183
:1064C000AF919F918F917F916F915F914F913F918C
:1064D0002F910F900FBE0F901F901895CF93DF93C1
:1064E000482F50E0CA018E5B9C4FFC013491425D05
:1064F0005C4FFA018491882369F190E0880F991F1D
:10650000FC01E05FFC4FA591B491FC01E65EFC4FFD
:10651000C591D491662351F42FB7F8948C91932FA1
:10652000909589238C93888189230BC0623061F414
:106530002FB7F8948C91932F909589238C93888111
:10654000832B88832FBF06C09FB7F8948C91832B31
:106550008C939FBFDF91CF910895482F50E0CA01DF
:106560008A5A9C4FFC012491CA018E5B9C4FFC010E
:106570009491425D5C4FFA013491332309F440C099
:10658000222351F1233071F0243028F42130A1F07E
:10659000223011F514C02630B1F02730C1F024307C
:1065A000D9F404C0809180008F7703C0809180006F
:1065B0008F7D8093800010C084B58F7702C084B532
:1065C0008F7D84BD09C08091B0008F7703C080911A
:1065D000B0008F7D8093B000E32FF0E0EE0FFF1F3F
:1065E000E65EFC4FA591B4912FB7F894662321F491
:1065F0008C919095892302C08C91892B8C932FBF0D
:106600000895CF92DF92EF92FF920F931F93CF9353
:10661000DF937C016B018A01C0E0D0E00FC0D6019E
:106620006D916D01D701ED91FC910190F081E02D0C
:10663000C7010995C80FD91F015010400115110558
:1066400071F7CE01DF91CF911F910F91FF90EF90E5
:10665000DF90CF900895CF93DF930E94D9310E94AD
:10666000CF27C0E0D0E00E94AF292097E1F30E943D
:106670000000F9CF5058BB27AA270ED041C201D243
:1066800030F006D220F031F49F3F11F41EF4C0C167
:106690000EF4E095E7FBB6C1E92F54D280F3BA17A8
:1066A000620773078407950718F071F49EF56CC2B2
:1066B0000EF4E0950B2EBA2FA02D0B01B90190011D
:1066C0000C01CA01A0011124FF27591B99F0593F61
:1066D00050F4503E68F11A16F040A22F232F342FA9
:1066E0004427585FF3CF469537952795A795F040F7
:1066F0005395C9F77EF41F16BA0B620B730B840B0C
:10670000BAF09150A1F0FF0FBB1F661F771F881FC3
:10671000C2F70EC0BA0F621F731F841F48F487951B
:1067200077956795B795F7959E3F08F0B3CF93950A
:10673000880F08F09927EE0F979587950895A1D1B6
:1067400058F080E891E009F49EEFA2D128F040E8EB
:1067500051E059F45EEF09C05BC116C2E92FE07841
:10676000F1D168F3092E052AC1F326173707480728
:10677000590738F00E2E07F8E02569F0E025E064AF
:106780000AC0EF6307F8009407FADB01B9019D0125
:10679000DC01CA01AD01EF934AD0B2D10AD05F91BA
:1067A000552331F02BED3FE049E450FD49EC63CF38
:1067B0000895DF93DD27B92FBF7740E85FE3161612
:1067C000170648075B0710F4D92FE9D19F938F93E1
:1067D0007F936F93BCD2E8E6F0E01DD191D12F9169
:1067E0003F914F915F91EED1DD2349F09058A2EA9D
:1067F0002AED3FE049EC5FE3D0785D274DDFDF9184
:106800007FC1DCD008F481E008954AD1E39589C1C5
:106810000CD076C13DD140F034D130F021F45F3F4F
:1068200019F0F0C05111B1C1F3C08CD198F3992384
:10683000C9F35523B1F3951B550BBB27AA27621744
:106840007307840738F09F5F5F4F220F331F441F89
:10685000AA1FA9F333D00E2E3AF0E0E830D09150C1
:106860005040E695001CCAF729D0FE2F27D0660FAE
:10687000771F881FBB1F261737074807AB07B0E8ED
:1068800009F0BB0B802DBF01FF2793585F4F2AF003
:106890009E3F510568F0B6C078C15F3FECF3983E6B
:1068A000DCF3869577956795B795F7959F5FC9F760
:1068B000880F911D9695879597F90895E1E0660FE9
:1068C000771F881FBB1F621773078407BA0720F062
:1068D000621B730B840BBA0BEE1F88F7E0950895CB
:1068E00004D06894B11151C1089534D188F09F57F4
:1068F00090F0B92F9927B751A0F0D1F0660F771F0C
:10690000881F991F1AF0BA95C9F712C0B13081F0EB
:106910003BD1B1E0089538C1672F782F8827B85F41
:1069200039F0B93FCCF3869577956795B395D9F74C
:106930003EF490958095709561957F4F8F4F9F4F56
:106940000895E89409C097FB3EF490958095709562
:1069500061957F4F8F4F9F4F9923A9F0F92F96E9AB
:10696000BB279395F695879577956795B795F11120
:10697000F8CFFAF4BB0F11F460FF1BC06F5F7F4FBD
:106980008F4F9F4F16C0882311F096E911C07723CF
:1069900021F09EE8872F762F05C0662371F096E8D8
:1069A000862F70E060E02AF09A95660F771F881FA7
:1069B000DAF7880F9695879597F90895990F00084B
:1069C000550FAA0BE0E8FEEF16161706E807F907C1
:1069D000C0F012161306E407F50798F0621B730B5C
:1069E000840B950B39F40A2661F0232B242B252BDD
:1069F00021F408950A2609F4A140A6958FEF811D80
:106A0000811D089597F99F6780E870E060E0089520
:106A10009FEF80EC0895DF93CF931F930F93FF9226
:106A2000EF92DF927B018C01689405C0DA2EEF01B2
:106A3000C9D0FE01E894A5912591359145915591D4
:106A4000AEF3EF0129DEFE019701A801DA9479F790
:106A5000DF90EF90FF900F911F91CF91DF910895FC
:106A60009F938F937F936F93FF93EF939B01AC0161
:106A70009DD0EF91FF91CFDF2F913F914F915F918B
:106A800095C000240A9416161706180609060895DC
:106A900000240A9412161306140605060895B8CFAA
:106AA00059D0E8F3E894EFEFBB273FE048EC5FE70D
:106AB0006B3D73078407950708F1FF279F57B25A6C
:106AC0006A4D7F40894CF04032F4BE556542704FAC
:106AD0008643FF4F0894EE1F915030F0BB0F661FA6
:106AE000771F881FFF1FEBCF9EE7882332F0BB0F75
:106AF000661F771F881F9A95C1F79395E09565C12A
:106B0000092E0394000C11F4882352F0BB0F40F4BB
:106B1000BF2B11F460FF04C06F5F7F4F8F4F9F4FFB
:106B20000895EF93E0FF06C0A2EA2AED3FE049ECAA
:106B30005FEBB2DDE5DF0F90039401FC9058E5E9CF
:106B4000F0E08ECF57FD9058440F551F59F05F3F2E
:106B500071F04795880F97FB991F61F09F3F79F07F
:106B600087950895121613061406551FF2CF469501
:106B7000F1DF08C0161617061806991FF1CF869583
:106B80007105610508940895E894BB276627772767
:106B9000CB0197F9089512DF08F48FEF08959B0158
:106BA000AC0160E070E080E89FE332CE0BD0A8CF6C
:106BB00068DF28F06DDF18F0952309F023CF28CF88
:106BC0001124E3CFBFDFA0F3959FD1F3950F50E0E1
:106BD000551F629FF001729FBB27F00DB11D639F8F
:106BE000AA27F00DB11DAA1F649F6627B00DA11D35
:106BF000661F829F2227B00DA11D621F739FB00DDB
:106C0000A11D621F839FA00D611D221F749F33274A
:106C1000A00D611D231F849F600D211D822F762FE3
:106C20006A2F11249F5750408AF0E1F088234AF0E0
:106C3000EE0FFF1FBB1F661F771F881F915050402C
:106C4000A9F79E3F510570F0DDCE9FCF5F3FECF37B
:106C5000983EDCF3869577956795B795F795E79518
:106C60009F5FC1F7FE2B880F911D9695879597F929
:106C7000089570DFE0F09E37D8F09639B8F49E386A
:106C800048F4672F782F8827985FF9CF86957795F6
:106C9000679593959539D0F3B62FB1706B0F711D31
:106CA000811D20F4879577956795939573C08DC066
:106CB0006CCF11F40EF4ACCE88C04CDFD0F3992326
:106CC000D9F3CEF39F57550B87FF8FD056959795E5
:106CD000B0E020F4660F771F881FBB1F1F930F9330
:106CE00000249001A0018001F001A0E80E0F1F1FF9
:106CF0000A1E511D601B710B8009B50B48F4600F13
:106D0000711F801DB51F0E1B1F0B0A0A510907C0FA
:106D10002E0F3F1F4A1F0E0F1F1F0A1E511D660F09
:106D2000771F881FBB1FA695F795E795F8F60617FE
:106D3000170708065B07211D311D411D0F911F918B
:106D4000B901842F9158880F9695879508959B01D6
:106D5000AC012CCFDF93D92FA3DEE695D7952AED92
:106D60003FE049E45FE3B33A62077307840795079E
:106D7000D7952AF0A2EA49EC90688EDCC1DEE3EBFD
:106D8000F0E06EDEDD0F0BF00ADFDD0F0BF4905844
:106D9000DF910895882371F4772321F09850872B91
:106DA000762F07C0662311F499270DC09051862BCA
:106DB00070E060E02AF09A95660F771F881FDAF777
:106DC000880F9695879597F908959F3F49F09150C0
:106DD00028F4869577956795B7959F5F80389F4F84
:106DE000880F9695879597F9089591505040660FB2
:106DF000771F881FD2F70895AA1BBB1B51E107C05C
:106E0000AA1FBB1FA617B70710F0A61BB70B881F3A
:106E1000991F5A95A9F780959095BC01CD010895C9
:106E200097FB092E07260AD077FD04D0E5DF06D0B0
:106E300000201AF4709561957F4F0895F6F79095AC
:106E400081959F4F0895A1E21A2EAA1BBB1BFD013D
:106E50000DC0AA1FBB1FEE1FFF1FA217B307E40739
:106E6000F50720F0A21BB30BE40BF50B661F771F91
:106E7000881F991F1A9469F7609570958095909571
:106E80009B01AC01BD01CF01089597FB092E05269A
:106E90000ED057FD04D0D7DF0AD0001C38F450952F
:106EA0004095309521953F4F4F4F5F4F0895F6F72E
:106EB00090958095709561957F4F8F4F9F4F089566
:106EC000EE0FFF1F0590F491E02D0994F894FFCF89
:106ED0002563002563256300256325326925632525
:106EE0003032697C2563253269256325303269009B
:106EF00025632532692563253032690025352E301A
:106F000066256300256325312E35662563002563DC
:106F1000253569256300256325352E3266256300F6
:106F20006D616E00737431007374320073743300DA
:106F30007374340073743500737436007068200005
:106F4000636C200076722000686C20006170200065
:106F5000727462006C616E0070702000706F690066
:106F600061632000006174200025632573002563A0
:106F700025332E3069256300253469256325630098
:106F8000256325336925630025737C2563257325D7
:106F9000630020C0C0C0C0C0C7C0C0C0C0C0200007
:106FA00025342E3066256300256325332E30662573
:106FB0006300256325352E30662563002563253162
:106FC000312E36667C25632531312E3666002563E9
:106FD0002532690025332E316625630020202020CC
:106FE000202020202020202000202064697361724E
:106FF0006D6564202000206E6F2074656C20636FC7
:107000006D2000206E6F2067707320666978200005
:1070100062617474207761726E696E670062617478
:1070200074637269746963616C00206261747420B6
:107030006572726F7220006C696E6B207175616C85
:10704000697479006D6167207761726E696E67009F
:107050006D616720637269746963616C00206D61A2
:107060006720206572726F7220002573002000B4C3
:10707000060000E803E803E803E8039DFF0164005D
:1070800000000077050133750478047B047E04BB9F
:107090002900070E091C1B1215383F363124232AFC
:1070A0002D70777E796C6B6265484F464154535A18
:1070B0005DE0E7EEE9FCFBF2F5D8DFD6D1C4C3CA48
:1070C000CD90979E998C8B8285A8AFA6A1B4B3BAB8
:1070D000BDC7C0C9CEDBDCD5D2FFF8F1F6E3E4EDE5
:1070E000EAB7B0B9BEABACA5A28F88818693949D58
:1070F0009A2720292E3B3C35321F18111603040D08
:107100000A5750595E4B4C45426F68616673747DF7
:107110007A898E878095929B9CB1B6BFB8ADAAA3A1
:10712000A4F9FEF7F0E5E2EBECC1C6CFC8DDDAD397
:10713000D4696E676075727B7C51565F584D4A43C7
:1071400044191E171005020B0C21262F283D3A3337
:10715000344E49404752555C5B7671787F6A6D6466
:10716000633E39303722252C2B0601080F1A1D14D7
:1071700013AEA9A0A7B2B5BCBB9691989F8A8D8487
:1071800083DED9D0D7C2C5CCCBE6E1E8EFFAFDF477
:10719000F3C2C0C0C1C0C0C1C0C0C4C0C0C1C0C0B3
:1071A000C1C0C0C3C0C0C1C0C0C1C0C0C5C0C0C1D3
:1071B000C0C0C1C0C000000000D12A0133422A7201
:0E71C0002AA22ABF2A582AE029262B962B0045
:00000001FF
